 attach009Agent00

 Timestamp is 4fcb293d (reproducible build file hash)

 Preferred load address is 0000000180000000

 Start         Length     Name                   Class
 0001:00000000 00003cc0H .text$mn                CODE
 0001:00003cc0 00000036H .text$mn$00             CODE
 0001:00003cf6 00000092H .text$x                 CODE
 0002:00000000 000001b8H .idata$5                DATA
 0002:000001b8 00000038H .00cfg                  DATA
 0002:000001f0 00000008H .CRT$XCA                DATA
 0002:000001f8 00000008H .CRT$XCZ                DATA
 0002:00000200 00000008H .CRT$XIA                DATA
 0002:00000208 00000008H .CRT$XIC                DATA
 0002:00000210 00000008H .CRT$XIZ                DATA
 0002:00000218 00000008H .CRT$XLA                DATA
 0002:00000220 00000008H .CRT$XLZ                DATA
 0002:00000228 00000008H .CRT$XPA                DATA
 0002:00000230 00000008H .CRT$XPZ                DATA
 0002:00000238 00000008H .CRT$XTA                DATA
 0002:00000240 00000010H .CRT$XTZ                DATA
 0002:00000248 00000000H .gehcont$y              DATA
 0002:00000248 00000000H .gfids$y                DATA
 0002:00000250 00002530H .rdata                  DATA
 0002:00002780 00000000H .rdata$CastGuardVftablesA DATA
 0002:00002780 00000000H .rdata$CastGuardVftablesC DATA
 0002:00002780 00000028H .rdata$T                DATA
 0002:000027a8 000000b8H .rdata$voltmd           DATA
 0002:00002860 00000320H .rdata$zzzdbg           DATA
 0002:00002b80 00000008H .rtc$IAA                DATA
 0002:00002b88 00000008H .rtc$IZZ                DATA
 0002:00002b90 00000008H .rtc$TAA                DATA
 0002:00002b98 00000008H .rtc$TZZ                DATA
 0002:00002ba0 00000004H .tls                    DATA
 0002:00002ba4 00000004H .tls$                   DATA
 0002:00002ba8 00000008H .tls$ZZZ                DATA
 0002:00002bb0 000003c0H .xdata                  DATA
 0002:00002f70 00000354H .edata                  DATA
 0002:000032c4 00000078H .idata$2                DATA
 0002:0000333c 00000014H .idata$3                DATA
 0002:00003350 000001b8H .idata$4                DATA
 0002:00003508 0000045aH .idata$6                DATA
 0003:00000000 000000a0H .data                   DATA
 0003:000000a0 0001b708H .bss                    DATA
 0004:00000000 0000042cH .pdata                  DATA

  Address         Publics by Value              Rva+Base               Lib:Object

 0000:00000000       __AbsoluteZero             0000000000000000     <absolute>
 0000:00000000       ___safe_se_handler_count   0000000000000000     <absolute>
 0000:00000000       ___safe_se_handler_table   0000000000000000     <absolute>
 0000:00000000       __arm64x_extra_rfe_table   0000000000000000     <absolute>
 0000:00000000       __arm64x_extra_rfe_table_size 0000000000000000     <absolute>
 0000:00000000       __arm64x_native_entrypoint 0000000000000000     <absolute>
 0000:00000000       __arm64x_redirection_metadata 0000000000000000     <absolute>
 0000:00000000       __arm64x_redirection_metadata_count 0000000000000000     <absolute>
 0000:00000000       __dynamic_value_reloc_table 0000000000000000     <absolute>
 0000:00000000       __enclave_config           0000000000000000     <absolute>
 0000:00000000       __guard_check_icall_a64n_fptr 0000000000000000     <absolute>
 0000:00000000       __guard_eh_cont_count      0000000000000000     <absolute>
 0000:00000000       __guard_eh_cont_table      0000000000000000     <absolute>
 0000:00000000       __guard_fids_count         0000000000000000     <absolute>
 0000:00000000       __guard_fids_table         0000000000000000     <absolute>
 0000:00000000       __guard_iat_count          0000000000000000     <absolute>
 0000:00000000       __guard_iat_table          0000000000000000     <absolute>
 0000:00000000       __guard_longjmp_count      0000000000000000     <absolute>
 0000:00000000       __guard_longjmp_table      0000000000000000     <absolute>
 0000:00000000       __hybrid_auxiliary_iat     0000000000000000     <absolute>
 0000:00000000       __hybrid_auxiliary_iat_copy 0000000000000000     <absolute>
 0000:00000000       __hybrid_code_map          0000000000000000     <absolute>
 0000:00000000       __hybrid_code_map_count    0000000000000000     <absolute>
 0000:00000000       __x64_code_ranges_to_entry_points 0000000000000000     <absolute>
 0000:00000000       __x64_code_ranges_to_entry_points_count 0000000000000000     <absolute>
 0000:00000100       __guard_flags              0000000000000100     <absolute>
 0000:00000000       __ImageBase                0000000180000000     <linker-defined>
 0001:00000000       ?CallStaticVoidMethod@JNIEnv_@@QEAAXPEAV_jclass@@PEAU_jmethodID@@ZZ 0000000180001000 f i libattach009Agent00.obj
 0001:00000024       ?NewObject@JNIEnv_@@QEAAPEAV_jobject@@PEAV_jclass@@PEAU_jmethodID@@ZZ 0000000180001024 f i libattach009Agent00.obj
 0001:0000004c       ?SetEventNotificationMode@_jvmtiEnv@@QEAA?AW4jvmtiError@@W4jvmtiEventMode@@W4jvmtiEvent@@PEAV_jobject@@ZZ 000000018000104c f i libattach009Agent00.obj
 0001:00000058       ?TranslateError@@YAPEBDW4jvmtiError@@@Z 0000000180001058 f   libattach009Agent00.obj
 0001:00000310       ?nsk_jni_check_exception@@YAHPEAUJNIEnv_@@QEBDH@Z 0000000180001310 f   libattach009Agent00.obj
 0001:00000454       ?nsk_jni_lverify@@YAHHPEAUJNIEnv_@@HQEBDH1ZZ 0000000180001454 f   libattach009Agent00.obj
 0001:000004f4       Agent_OnAttach             00000001800014f4 f   libattach009Agent00.obj
 0001:00000778       Java_nsk_jvmti_unit_FollowReferences_FollowRefObjects_addRefToVerify 0000000180001778 f   libattach009Agent00.obj
 0001:00000950       Java_nsk_jvmti_unit_FollowReferences_FollowRefObjects_getTag 0000000180001950 f   libattach009Agent00.obj
 0001:00000a10       Java_nsk_jvmti_unit_FollowReferences_FollowRefObjects_resetRefsToVerify 0000000180001a10 f   libattach009Agent00.obj
 0001:00000a18       Java_nsk_jvmti_unit_FollowReferences_FollowRefObjects_resetTags 0000000180001a18 f   libattach009Agent00.obj
 0001:00000a5c       Java_nsk_jvmti_unit_FollowReferences_FollowRefObjects_setTag 0000000180001a5c f   libattach009Agent00.obj
 0001:00000cb4       Java_nsk_share_jvmti_ArgumentHandler_getAgentOptionsString 0000000180001cb4 f   libattach009Agent00.obj
 0001:00000d64       Java_nsk_share_jvmti_DebugeeClass_checkStatus 0000000180001d64 f   libattach009Agent00.obj
 0001:00000dec       Java_nsk_share_jvmti_DebugeeClass_resetAgentData 0000000180001dec f   libattach009Agent00.obj
 0001:00000e4c       Java_nsk_share_jvmti_RedefineAgent_agentStatus 0000000180001e4c f   libattach009Agent00.obj
 0001:00000e58       Java_nsk_share_jvmti_RedefineAgent_isRedefined 0000000180001e58 f   libattach009Agent00.obj
 0001:00000e64       Java_nsk_share_jvmti_RedefineAgent_redefineAttempted 0000000180001e64 f   libattach009Agent00.obj
 0001:00000e70       MA_checkStatus             0000000180001e70 f   libattach009Agent00.obj
 0001:00000f14       __local_stdio_printf_options 0000000180001f14 f i libattach009Agent00.obj
 0001:000010f4       classLoadHandler           00000001800020f4 f   libattach009Agent00.obj
 0001:00001364       exitOnError                0000000180002364 f   libattach009Agent00.obj
 0001:00001418       fprintf                    0000000180002418 f i libattach009Agent00.obj
 0001:0000145c       nsk_aod_agentFinished      000000018000245c f   libattach009Agent00.obj
 0001:00001658       nsk_aod_agentLoaded        0000000180002658 f   libattach009Agent00.obj
 0001:00001928       nsk_aod_createJNIEnv       0000000180002928 f   libattach009Agent00.obj
 0001:000019a0       nsk_aod_createOptions      00000001800029a0 f   libattach009Agent00.obj
 0001:00001c10       nsk_aod_getOptionValue     0000000180002c10 f   libattach009Agent00.obj
 0001:00001cfc       nsk_aod_internal_error     0000000180002cfc f   libattach009Agent00.obj
 0001:00001d28       nsk_aod_optionSpecified    0000000180002d28 f   libattach009Agent00.obj
 0001:00001df0       nsk_free_options           0000000180002df0 f   libattach009Agent00.obj
 0001:00001e50       nsk_jvmti_aod_deallocate   0000000180002e50 f   libattach009Agent00.obj
 0001:00001f08       nsk_jvmti_aod_disableEventAndFinish 0000000180002f08 f   libattach009Agent00.obj
 0001:00001fc0       nsk_jvmti_aod_getClassName 0000000180002fc0 f   libattach009Agent00.obj
 0001:000020a0       nsk_jvmti_aod_getThreadName 00000001800030a0 f   libattach009Agent00.obj
 0001:00002184       nsk_jvmti_createJVMTIEnv   0000000180003184 f   libattach009Agent00.obj
 0001:000022b4       nsk_jvmti_lverify          00000001800032b4 f   libattach009Agent00.obj
 0001:000023a4       nsk_jvmti_resetAgentData   00000001800033a4 f   libattach009Agent00.obj
 0001:00002424       nsk_jvmti_setFailStatus    0000000180003424 f   libattach009Agent00.obj
 0001:00002460       nsk_lcomplain              0000000180003460 f   libattach009Agent00.obj
 0001:00002480       nsk_ldisplay               0000000180003480 f   libattach009Agent00.obj
 0001:000024a0       nsk_ltrace                 00000001800034a0 f   libattach009Agent00.obj
 0001:000024c0       nsk_lvcomplain             00000001800034c0 f   libattach009Agent00.obj
 0001:00002678       nsk_lvdisplay              0000000180003678 f   libattach009Agent00.obj
 0001:000026c4       nsk_lverify                00000001800036c4 f   libattach009Agent00.obj
 0001:00002720       nsk_lvtrace                0000000180003720 f   libattach009Agent00.obj
 0001:00002780       nsk_printf                 0000000180003780 f   libattach009Agent00.obj
 0001:000027a8       nsk_vprintf                00000001800037a8 f   libattach009Agent00.obj
 0001:0000285c       printf                     000000018000385c f i libattach009Agent00.obj
 0001:00002d84       __raise_securityfailure    0000000180003d84 f   MSVCRT:gs_report.obj
 0001:00002db8       __report_gsfailure         0000000180003db8 f   MSVCRT:gs_report.obj
 0001:00002ff8       __GSHandlerCheck           0000000180003ff8 f   MSVCRT:gshandler.obj
 0001:00003018       __GSHandlerCheckCommon     0000000180004018 f   MSVCRT:gshandler.obj
 0001:00003090       __security_check_cookie    0000000180004090 f   MSVCRT:amdsecgs.obj
 0001:000033d0       _DllMainCRTStartup         00000001800043d0 f   MSVCRT:dll_dllmain.obj
 0001:00003410       __scrt_acquire_startup_lock 0000000180004410 f   MSVCRT:utility.obj
 0001:0000344c       __scrt_dllmain_after_initialize_c 000000018000444c f   MSVCRT:utility.obj
 0001:00003480       __scrt_dllmain_before_initialize_c 0000000180004480 f   MSVCRT:utility.obj
 0001:00003498       __scrt_dllmain_crt_thread_attach 0000000180004498 f   MSVCRT:utility.obj
 0001:000034c0       __scrt_dllmain_crt_thread_detach 00000001800044c0 f   MSVCRT:utility.obj
 0001:000034d8       __scrt_dllmain_exception_filter 00000001800044d8 f   MSVCRT:utility.obj
 0001:00003538       __scrt_dllmain_uninitialize_c 0000000180004538 f   MSVCRT:utility.obj
 0001:00003568       __scrt_dllmain_uninitialize_critical 0000000180004568 f   MSVCRT:utility.obj
 0001:0000357c       __scrt_initialize_crt      000000018000457c f   MSVCRT:utility.obj
 0001:000035c8       __scrt_initialize_onexit_tables 00000001800045c8 f   MSVCRT:utility.obj
 0001:00003654       __scrt_is_nonwritable_in_current_image 0000000180004654 f   MSVCRT:utility.obj
 0001:000036ec       __scrt_release_startup_lock 00000001800046ec f   MSVCRT:utility.obj
 0001:00003710       __scrt_uninitialize_crt    0000000180004710 f   MSVCRT:utility.obj
 0001:0000373c       _onexit                    000000018000473c f   MSVCRT:utility.obj
 0001:00003778       atexit                     0000000180004778 f   MSVCRT:utility.obj
 0001:00003790       __crt_debugger_hook        0000000180004790 f   MSVCRT:utility_desktop.obj
 0001:00003798       __scrt_fastfail            0000000180004798 f   MSVCRT:utility_desktop.obj
 0001:000038e4       _guard_check_icall_nop     00000001800048e4 f i MSVCRT:guard_support.obj
 0001:000038e8       __security_init_cookie     00000001800048e8 f   MSVCRT:gs_support.obj
 0001:00003994       DllMain                    0000000180004994 f   MSVCRT:dll_dllmain_stub.obj
 0001:000039b8       ?__scrt_initialize_type_info@@YAXXZ 00000001800049b8 f   MSVCRT:tncleanup.obj
 0001:000039c8       ?__scrt_uninitialize_type_info@@YAXXZ 00000001800049c8 f   MSVCRT:tncleanup.obj
 0001:000039d4       __local_stdio_scanf_options 00000001800049d4 f i MSVCRT:default_local_stdio_options.obj
 0001:000039dc       __scrt_initialize_default_local_stdio_options 00000001800049dc f   MSVCRT:default_local_stdio_options.obj
 0001:000039f8       __scrt_get_dyn_tls_init_callback 00000001800049f8 f   MSVCRT:dyn_tls_init.obj
 0001:00003a00       _RTC_Initialize            0000000180004a00 f   MSVCRT:initsect.obj
 0001:00003a3c       _RTC_Terminate             0000000180004a3c f   MSVCRT:initsect.obj
 0001:00003a78       __isa_available_init       0000000180004a78 f   MSVCRT:cpu_disp.obj
 0001:00003c24       _get_startup_argv_mode     0000000180004c24 f   MSVCRT:argv_mode.obj
 0001:00003c2c       __scrt_is_ucrt_dll_in_use  0000000180004c2c f   MSVCRT:ucrt_detection.obj
 0001:00003c40       memcpy                     0000000180004c40 f   vcruntime:VCRUNTIME140.dll
 0001:00003c46       memset                     0000000180004c46 f   vcruntime:VCRUNTIME140.dll
 0001:00003c4c       strchr                     0000000180004c4c f   vcruntime:VCRUNTIME140.dll
 0001:00003c52       __C_specific_handler       0000000180004c52 f   vcruntime:VCRUNTIME140.dll
 0001:00003c58       __std_type_info_destroy_list 0000000180004c58 f   vcruntime:VCRUNTIME140.dll
 0001:00003c5e       strcmp                     0000000180004c5e f   ucrt:api-ms-win-crt-string-l1-1-0.dll
 0001:00003c64       strcpy                     0000000180004c64 f   ucrt:api-ms-win-crt-string-l1-1-0.dll
 0001:00003c6a       strlen                     0000000180004c6a f   ucrt:api-ms-win-crt-string-l1-1-0.dll
 0001:00003c70       _initterm                  0000000180004c70 f   ucrt:api-ms-win-crt-runtime-l1-1-0.dll
 0001:00003c76       _initterm_e                0000000180004c76 f   ucrt:api-ms-win-crt-runtime-l1-1-0.dll
 0001:00003c7c       _seh_filter_dll            0000000180004c7c f   ucrt:api-ms-win-crt-runtime-l1-1-0.dll
 0001:00003c82       _configure_narrow_argv     0000000180004c82 f   ucrt:api-ms-win-crt-runtime-l1-1-0.dll
 0001:00003c88       _initialize_narrow_environment 0000000180004c88 f   ucrt:api-ms-win-crt-runtime-l1-1-0.dll
 0001:00003c8e       _initialize_onexit_table   0000000180004c8e f   ucrt:api-ms-win-crt-runtime-l1-1-0.dll
 0001:00003c94       _register_onexit_function  0000000180004c94 f   ucrt:api-ms-win-crt-runtime-l1-1-0.dll
 0001:00003c9a       _execute_onexit_table      0000000180004c9a f   ucrt:api-ms-win-crt-runtime-l1-1-0.dll
 0001:00003ca0       _crt_atexit                0000000180004ca0 f   ucrt:api-ms-win-crt-runtime-l1-1-0.dll
 0001:00003ca6       _cexit                     0000000180004ca6 f   ucrt:api-ms-win-crt-runtime-l1-1-0.dll
 0001:00003cac       __acrt_initialize          0000000180004cac f   MSVCRT:ucrt_stubs.obj
 0001:00003cac       __acrt_thread_attach       0000000180004cac f   MSVCRT:ucrt_stubs.obj
 0001:00003cac       __acrt_thread_detach       0000000180004cac f   MSVCRT:ucrt_stubs.obj
 0001:00003cac       __acrt_uninitialize        0000000180004cac f   MSVCRT:ucrt_stubs.obj
 0001:00003cac       __acrt_uninitialize_critical 0000000180004cac f   MSVCRT:ucrt_stubs.obj
 0001:00003cac       __scrt_stub_for_acrt_initialize 0000000180004cac f   MSVCRT:ucrt_stubs.obj
 0001:00003cac       __scrt_stub_for_acrt_thread_attach 0000000180004cac f   MSVCRT:ucrt_stubs.obj
 0001:00003cac       __scrt_stub_for_acrt_thread_detach 0000000180004cac f   MSVCRT:ucrt_stubs.obj
 0001:00003cac       __scrt_stub_for_acrt_uninitialize 0000000180004cac f   MSVCRT:ucrt_stubs.obj
 0001:00003cac       __scrt_stub_for_acrt_uninitialize_critical 0000000180004cac f   MSVCRT:ucrt_stubs.obj
 0001:00003cac       __vcrt_initialize          0000000180004cac f   MSVCRT:ucrt_stubs.obj
 0001:00003cac       __vcrt_thread_attach       0000000180004cac f   MSVCRT:ucrt_stubs.obj
 0001:00003cac       __vcrt_thread_detach       0000000180004cac f   MSVCRT:ucrt_stubs.obj
 0001:00003cac       __vcrt_uninitialize        0000000180004cac f   MSVCRT:ucrt_stubs.obj
 0001:00003cac       __vcrt_uninitialize_critical 0000000180004cac f   MSVCRT:ucrt_stubs.obj
 0001:00003cb0       __scrt_stub_for_is_c_termination_complete 0000000180004cb0 f   MSVCRT:ucrt_stubs.obj
 0001:00003cb0       _is_c_termination_complete 0000000180004cb0 f   MSVCRT:ucrt_stubs.obj
 0001:00003cd0       _guard_dispatch_icall_nop  0000000180004cd0 f   MSVCRT:guard_dispatch.obj
 0001:00003cf0       _guard_xfg_dispatch_icall_nop 0000000180004cf0 f   MSVCRT:guard_xfg_dispatch.obj
 0002:00000000       __imp_RtlCaptureContext    0000000180005000     kernel32:KERNEL32.dll
 0002:00000008       __imp_RtlLookupFunctionEntry 0000000180005008     kernel32:KERNEL32.dll
 0002:00000010       __imp_RtlVirtualUnwind     0000000180005010     kernel32:KERNEL32.dll
 0002:00000018       __imp_UnhandledExceptionFilter 0000000180005018     kernel32:KERNEL32.dll
 0002:00000020       __imp_SetUnhandledExceptionFilter 0000000180005020     kernel32:KERNEL32.dll
 0002:00000028       __imp_GetCurrentProcess    0000000180005028     kernel32:KERNEL32.dll
 0002:00000030       __imp_TerminateProcess     0000000180005030     kernel32:KERNEL32.dll
 0002:00000038       __imp_IsProcessorFeaturePresent 0000000180005038     kernel32:KERNEL32.dll
 0002:00000040       __imp_CloseHandle          0000000180005040     kernel32:KERNEL32.dll
 0002:00000048       __imp_InitializeCriticalSectionAndSpinCount 0000000180005048     kernel32:KERNEL32.dll
 0002:00000050       __imp_DeleteCriticalSection 0000000180005050     kernel32:KERNEL32.dll
 0002:00000058       __imp_CreateEventW         0000000180005058     kernel32:KERNEL32.dll
 0002:00000060       __imp_GetModuleHandleW     0000000180005060     kernel32:KERNEL32.dll
 0002:00000068       __imp_GetProcAddress       0000000180005068     kernel32:KERNEL32.dll
 0002:00000070       __imp_IsDebuggerPresent    0000000180005070     kernel32:KERNEL32.dll
 0002:00000078       __imp_QueryPerformanceCounter 0000000180005078     kernel32:KERNEL32.dll
 0002:00000080       __imp_GetCurrentProcessId  0000000180005080     kernel32:KERNEL32.dll
 0002:00000088       __imp_GetCurrentThreadId   0000000180005088     kernel32:KERNEL32.dll
 0002:00000090       __imp_GetSystemTimeAsFileTime 0000000180005090     kernel32:KERNEL32.dll
 0002:00000098       __imp_DisableThreadLibraryCalls 0000000180005098     kernel32:KERNEL32.dll
 0002:000000a0       __imp_InitializeSListHead  00000001800050a0     kernel32:KERNEL32.dll
 0002:000000a8       \177KERNEL32_NULL_THUNK_DATA 00000001800050a8     kernel32:KERNEL32.dll
 0002:000000b0       __imp_memcpy               00000001800050b0     vcruntime:VCRUNTIME140.dll
 0002:000000b8       __imp_memset               00000001800050b8     vcruntime:VCRUNTIME140.dll
 0002:000000c0       __imp_strchr               00000001800050c0     vcruntime:VCRUNTIME140.dll
 0002:000000c8       __imp___C_specific_handler 00000001800050c8     vcruntime:VCRUNTIME140.dll
 0002:000000d0       __imp___std_type_info_destroy_list 00000001800050d0     vcruntime:VCRUNTIME140.dll
 0002:000000d8       \177VCRUNTIME140_NULL_THUNK_DATA 00000001800050d8     vcruntime:VCRUNTIME140.dll
 0002:000000e0       __imp_malloc               00000001800050e0     ucrt:api-ms-win-crt-heap-l1-1-0.dll
 0002:000000e8       __imp_free                 00000001800050e8     ucrt:api-ms-win-crt-heap-l1-1-0.dll
 0002:000000f0       \177api-ms-win-crt-heap-l1-1-0_NULL_THUNK_DATA 00000001800050f0     ucrt:api-ms-win-crt-heap-l1-1-0.dll
 0002:000000f8       __imp__errno               00000001800050f8     ucrt:api-ms-win-crt-runtime-l1-1-0.dll
 0002:00000100       __imp_exit                 0000000180005100     ucrt:api-ms-win-crt-runtime-l1-1-0.dll
 0002:00000108       __imp__cexit               0000000180005108     ucrt:api-ms-win-crt-runtime-l1-1-0.dll
 0002:00000110       __imp__crt_atexit          0000000180005110     ucrt:api-ms-win-crt-runtime-l1-1-0.dll
 0002:00000118       __imp__execute_onexit_table 0000000180005118     ucrt:api-ms-win-crt-runtime-l1-1-0.dll
 0002:00000120       __imp__register_onexit_function 0000000180005120     ucrt:api-ms-win-crt-runtime-l1-1-0.dll
 0002:00000128       __imp__initialize_onexit_table 0000000180005128     ucrt:api-ms-win-crt-runtime-l1-1-0.dll
 0002:00000130       __imp__initialize_narrow_environment 0000000180005130     ucrt:api-ms-win-crt-runtime-l1-1-0.dll
 0002:00000138       __imp__configure_narrow_argv 0000000180005138     ucrt:api-ms-win-crt-runtime-l1-1-0.dll
 0002:00000140       __imp__seh_filter_dll      0000000180005140     ucrt:api-ms-win-crt-runtime-l1-1-0.dll
 0002:00000148       __imp__initterm_e          0000000180005148     ucrt:api-ms-win-crt-runtime-l1-1-0.dll
 0002:00000150       __imp__initterm            0000000180005150     ucrt:api-ms-win-crt-runtime-l1-1-0.dll
 0002:00000158       \177api-ms-win-crt-runtime-l1-1-0_NULL_THUNK_DATA 0000000180005158     ucrt:api-ms-win-crt-runtime-l1-1-0.dll
 0002:00000160       __imp___acrt_iob_func      0000000180005160     ucrt:api-ms-win-crt-stdio-l1-1-0.dll
 0002:00000168       __imp_fflush               0000000180005168     ucrt:api-ms-win-crt-stdio-l1-1-0.dll
 0002:00000170       __imp___stdio_common_vsprintf 0000000180005170     ucrt:api-ms-win-crt-stdio-l1-1-0.dll
 0002:00000178       __imp___stdio_common_vfprintf 0000000180005178     ucrt:api-ms-win-crt-stdio-l1-1-0.dll
 0002:00000180       \177api-ms-win-crt-stdio-l1-1-0_NULL_THUNK_DATA 0000000180005180     ucrt:api-ms-win-crt-stdio-l1-1-0.dll
 0002:00000188       __imp_strcmp               0000000180005188     ucrt:api-ms-win-crt-string-l1-1-0.dll
 0002:00000190       __imp_strcpy               0000000180005190     ucrt:api-ms-win-crt-string-l1-1-0.dll
 0002:00000198       __imp__strdup              0000000180005198     ucrt:api-ms-win-crt-string-l1-1-0.dll
 0002:00000198       __imp_strdup               0000000180005198     ucrt:api-ms-win-crt-string-l1-1-0.dll
 0002:000001a0       __imp_strlen               00000001800051a0     ucrt:api-ms-win-crt-string-l1-1-0.dll
 0002:000001a8       __imp_strncpy              00000001800051a8     ucrt:api-ms-win-crt-string-l1-1-0.dll
 0002:000001b0       \177api-ms-win-crt-string-l1-1-0_NULL_THUNK_DATA 00000001800051b0     ucrt:api-ms-win-crt-string-l1-1-0.dll
 0002:000001b8       __guard_check_icall_fptr   00000001800051b8     MSVCRT:guard_support.obj
 0002:000001c0       __guard_xfg_check_icall_fptr 00000001800051c0     MSVCRT:guard_support.obj
 0002:000001c8       __guard_dispatch_icall_fptr 00000001800051c8     MSVCRT:guard_support.obj
 0002:000001d0       __guard_xfg_dispatch_icall_fptr 00000001800051d0     MSVCRT:guard_support.obj
 0002:000001d8       __guard_xfg_table_dispatch_icall_fptr 00000001800051d8     MSVCRT:guard_support.obj
 0002:000001e0       __castguard_check_failure_os_handled_fptr 00000001800051e0     MSVCRT:guard_support.obj
 0002:000001e8       __guard_memcpy_fptr        00000001800051e8     vcruntime:softmemtag.obj
 0002:000001f0       __xc_a                     00000001800051f0     MSVCRT:initializers.obj
 0002:000001f8       __xc_z                     00000001800051f8     MSVCRT:initializers.obj
 0002:00000200       __xi_a                     0000000180005200     MSVCRT:initializers.obj
 0002:00000210       __xi_z                     0000000180005210     MSVCRT:initializers.obj
 0002:00000218       __xl_a                     0000000180005218     MSVCRT:tlssup.obj
 0002:00000220       __xl_z                     0000000180005220     MSVCRT:tlssup.obj
 0002:00000228       __xp_a                     0000000180005228     MSVCRT:initializers.obj
 0002:00000230       __xp_z                     0000000180005230     MSVCRT:initializers.obj
 0002:00000238       __xt_a                     0000000180005238     MSVCRT:initializers.obj
 0002:00000240       __xt_z                     0000000180005240     MSVCRT:initializers.obj
 0002:00000250       ??_C@_0BG@IKDDPPGD@?$CILjava?1lang?1String?$DL?$CJV@ 0000000180005250     libattach009Agent00.obj
 0002:00000270       g_refKindStr               0000000180005270     libattach009Agent00.obj
 0002:00000420       ??_C@_09BPLDFGCI@unknown_0@ 0000000180005420     libattach009Agent00.obj
 0002:00000430       ??_C@_0BL@FPNMECJD@JVMTI_HEAP_REFERENCE_CLASS@ 0000000180005430     libattach009Agent00.obj
 0002:00000450       ??_C@_0BL@FKGKKLNM@JVMTI_HEAP_REFERENCE_FIELD@ 0000000180005450     libattach009Agent00.obj
 0002:00000470       ??_C@_0CD@CAEHCFJF@JVMTI_HEAP_REFERENCE_ARRAY_ELEM@ 0000000180005470     libattach009Agent00.obj
 0002:00000498       ??_C@_0CC@DNEBMCNK@JVMTI_HEAP_REFERENCE_CLASS_LOAD@ 0000000180005498     libattach009Agent00.obj
 0002:000004c0       ??_C@_0BN@CJMIPEBB@JVMTI_HEAP_REFERENCE_SIGNERS@ 00000001800054c0     libattach009Agent00.obj
 0002:000004e0       ??_C@_0CH@HBOIDPEB@JVMTI_HEAP_REFERENCE_PROTECTION@ 00000001800054e0     libattach009Agent00.obj
 0002:00000508       ??_C@_0BP@MDKGDGKL@JVMTI_HEAP_REFERENCE_INTERFACE@ 0000000180005508     libattach009Agent00.obj
 0002:00000528       ??_C@_0CC@JJMIHNJH@JVMTI_HEAP_REFERENCE_STATIC_FIE@ 0000000180005528     libattach009Agent00.obj
 0002:00000550       ??_C@_0CD@IDHEEGID@JVMTI_HEAP_REFERENCE_CONSTANT_P@ 0000000180005550     libattach009Agent00.obj
 0002:00000578       ??_C@_0CA@EFFCHNG@JVMTI_HEAP_REFERENCE_SUPERCLASS@ 0000000180005578     libattach009Agent00.obj
 0002:00000598       ??_C@_0L@PCDFHGCJ@unknown_11@ 0000000180005598     libattach009Agent00.obj
 0002:000005a8       ??_C@_0L@NJBICFOK@unknown_12@ 00000001800055a8     libattach009Agent00.obj
 0002:000005b8       ??_C@_0L@MAADBEKL@unknown_13@ 00000001800055b8     libattach009Agent00.obj
 0002:000005c8       ??_C@_0L@IPECICGM@unknown_14@ 00000001800055c8     libattach009Agent00.obj
 0002:000005d8       ??_C@_0L@JGFJLDCN@unknown_15@ 00000001800055d8     libattach009Agent00.obj
 0002:000005e8       ??_C@_0L@LNHEOAOO@unknown_16@ 00000001800055e8     libattach009Agent00.obj
 0002:000005f8       ??_C@_0L@KEGPNBKP@unknown_17@ 00000001800055f8     libattach009Agent00.obj
 0002:00000608       ??_C@_0L@CDPHMNGA@unknown_18@ 0000000180005608     libattach009Agent00.obj
 0002:00000618       ??_C@_0L@DKOMPMCB@unknown_19@ 0000000180005618     libattach009Agent00.obj
 0002:00000628       ??_C@_0L@OJGIPJDB@unknown_20@ 0000000180005628     libattach009Agent00.obj
 0002:00000638       ??_C@_0CA@KAOFNDEM@JVMTI_HEAP_REFERENCE_JNI_GLOBAL@ 0000000180005638     libattach009Agent00.obj
 0002:00000658       ??_C@_0CC@HPFAJBK@JVMTI_HEAP_REFERENCE_SYSTEM_CLA@ 0000000180005658     libattach009Agent00.obj
 0002:00000680       ??_C@_0BN@FDEGFOHC@JVMTI_HEAP_REFERENCE_MONITOR@ 0000000180005680     libattach009Agent00.obj
 0002:000006a0       ??_C@_0CB@HKIBCMAJ@JVMTI_HEAP_REFERENCE_STACK_LOCA@ 00000001800056a0     libattach009Agent00.obj
 0002:000006c8       ??_C@_0BP@EAACMMOE@JVMTI_HEAP_REFERENCE_JNI_LOCAL@ 00000001800056c8     libattach009Agent00.obj
 0002:000006e8       ??_C@_0BM@IJDEOGOE@JVMTI_HEAP_REFERENCE_THREAD@ 00000001800056e8     libattach009Agent00.obj
 0002:00000708       ??_C@_0BL@EDGPPKC@JVMTI_HEAP_REFERENCE_OTHER@ 0000000180005708     libattach009Agent00.obj
 0002:00000724       ??_C@_04BCJPDBDA@Code@     0000000180005724     libattach009Agent00.obj
 0002:00000730       ??_C@_0BA@OCLMCFKC@LineNumberTable@ 0000000180005730     libattach009Agent00.obj
 0002:00000740       ??_C@_0BD@CPAEPILC@LocalVariableTable@ 0000000180005740     libattach009Agent00.obj
 0002:00000758       ??_C@_0BH@NMBDNHBD@LocalVariableTypeTable@ 0000000180005758     libattach009Agent00.obj
 0002:00000770       ??_C@_0O@HIHEEDNJ@StackMapTable@ 0000000180005770     libattach009Agent00.obj
 0002:00000780       ??_C@_0CN@NKCKIIJI@nsk?1share?1aod?1TargetApplication@ 0000000180005780     libattach009Agent00.obj
 0002:000007b0       ??_C@_0M@OANFKLGH@agentLoaded@ 00000001800057b0     libattach009Agent00.obj
 0002:000007c0       ??_C@_0O@JINEPNAJ@agentFinished@ 00000001800057c0     libattach009Agent00.obj
 0002:000007d0       ??_C@_0BH@BOPHNJNA@?$CILjava?1lang?1String?$DLZ?$CJV@ 00000001800057d0     libattach009Agent00.obj
 0002:000007e8       ??_C@_0L@HCDIAMJG@?9?5?$CFs?0?5?$CFd?3?5@ 00000001800057e8     libattach009Agent00.obj
 0002:00000800       ??_C@_0JI@HLPECLFI@?$CD?5?4?4?4?6?$CD?5ERROR?3?5too?5many?5complai@ 0000000180005800     libattach009Agent00.obj
 0002:000008a0       ??_C@_0ED@JNEKCCOB@The?5following?5fake?5exception?5st@ 00000001800058a0     libattach009Agent00.obj
 0002:000008e8       ??_C@_0CN@FCNMDFBH@nsk?4share?4Fake_Exception_for_RU@ 00000001800058e8     libattach009Agent00.obj
 0002:00000918       ??_C@_08PGFFNAEI@?$CI?$CFs?3?$CFd?$CJ?5@ 0000000180005918     libattach009Agent00.obj
 0002:00000928       ??_C@_0DP@IENMAEGI@s?2test?2hotspot?2jtreg?2vmTestbase@ 0000000180005928     libattach009Agent00.obj
 0002:00000968       ??_C@_0BL@NDJLFFJB@?7at?5nsk_lvcomplain?$CI?$CFs?3?$CFd?$CJ?6@ 0000000180005968     libattach009Agent00.obj
 0002:00000988       ??_C@_0BC@JOOKAFKF@?$CD?5ERROR?3?5?$CFs?0?5?$CFd?3?5@ 0000000180005988     libattach009Agent00.obj
 0002:000009a0       ??_C@_09KJEAHMEH@?$CD?5ERROR?3?5@ 00000001800059a0     libattach009Agent00.obj
 0002:000009ac       ??_C@_02GPIOPFAK@?$DO?$DO@ 00000001800059ac     libattach009Agent00.obj
 0002:000009b0       ??_C@_02FODMEDOG@?$DM?$DM@ 00000001800059b0     libattach009Agent00.obj
 0002:000009b4       ??_C@_02DJGKEECL@?4?4@     00000001800059b4     libattach009Agent00.obj
 0002:000009b8       ??_C@_0O@CJPGJOAF@?9?5?$CFs?0?5?$CFd?3?5?$CFs?5@ 00000001800059b8     libattach009Agent00.obj
 0002:000009c8       ??_C@_0CB@IAKPDOIC@?$CD?5?5?5verified?5assertion?5is?5FALSE@ 00000001800059c8     libattach009Agent00.obj
 0002:000009f0       ??_C@_0CO@LGONDEPD@stdout?3?5fflush?5failed?5?9?5err?$DN?$CFd?5@ 00000001800059f0     libattach009Agent00.obj
 0002:00000a20       ??_C@_0CO@KBGKJPBD@stderr?3?5fflush?5failed?5?9?5err?$DN?$CFd?5@ 0000000180005a20     libattach009Agent00.obj
 0002:00000a50       ??_C@_0BB@JCNMKLLK@JVMTI_ERROR_NONE@ 0000000180005a50     libattach009Agent00.obj
 0002:00000a68       ??_C@_0BL@LDIMKLPH@JVMTI_ERROR_INVALID_THREAD@ 0000000180005a68     libattach009Agent00.obj
 0002:00000a88       ??_C@_0CB@PJFPAIKJ@JVMTI_ERROR_INVALID_THREAD_GROU@ 0000000180005a88     libattach009Agent00.obj
 0002:00000ab0       ??_C@_0BN@LLMKHMNF@JVMTI_ERROR_INVALID_PRIORITY@ 0000000180005ab0     libattach009Agent00.obj
 0002:00000ad0       ??_C@_0CB@MBOFKAGB@JVMTI_ERROR_THREAD_NOT_SUSPENDE@ 0000000180005ad0     libattach009Agent00.obj
 0002:00000af8       ??_C@_0BN@FABOLPBI@JVMTI_ERROR_THREAD_SUSPENDED@ 0000000180005af8     libattach009Agent00.obj
 0002:00000b18       ??_C@_0BN@FDGNOBJM@JVMTI_ERROR_THREAD_NOT_ALIVE@ 0000000180005b18     libattach009Agent00.obj
 0002:00000b38       ??_C@_0BL@GOBIFKNJ@JVMTI_ERROR_INVALID_OBJECT@ 0000000180005b38     libattach009Agent00.obj
 0002:00000b58       ??_C@_0BK@FCMAJPPC@JVMTI_ERROR_INVALID_CLASS@ 0000000180005b58     libattach009Agent00.obj
 0002:00000b78       ??_C@_0BP@IKLLBKEB@JVMTI_ERROR_CLASS_NOT_PREPARED@ 0000000180005b78     libattach009Agent00.obj
 0002:00000b98       ??_C@_0BN@KLPPLKG@JVMTI_ERROR_INVALID_METHODID@ 0000000180005b98     libattach009Agent00.obj
 0002:00000bb8       ??_C@_0BN@BCEKOKND@JVMTI_ERROR_INVALID_LOCATION@ 0000000180005bb8     libattach009Agent00.obj
 0002:00000bd8       ??_C@_0BM@DFDGPME@JVMTI_ERROR_INVALID_FIELDID@ 0000000180005bd8     libattach009Agent00.obj
 0002:00000bf8       ??_C@_0BL@NELIEPEC@JVMTI_ERROR_NO_MORE_FRAMES@ 0000000180005bf8     libattach009Agent00.obj
 0002:00000c18       ??_C@_0BJ@BDBECFDM@JVMTI_ERROR_OPAQUE_FRAME@ 0000000180005c18     libattach009Agent00.obj
 0002:00000c38       ??_C@_0BK@MIIFNLOB@JVMTI_ERROR_TYPE_MISMATCH@ 0000000180005c38     libattach009Agent00.obj
 0002:00000c58       ??_C@_0BJ@HPCAOILC@JVMTI_ERROR_INVALID_SLOT@ 0000000180005c58     libattach009Agent00.obj
 0002:00000c78       ??_C@_0BG@CHILOPNI@JVMTI_ERROR_DUPLICATE@ 0000000180005c78     libattach009Agent00.obj
 0002:00000c90       ??_C@_0BG@DIEMLHKM@JVMTI_ERROR_NOT_FOUND@ 0000000180005c90     libattach009Agent00.obj
 0002:00000ca8       ??_C@_0BM@NHMCKHOB@JVMTI_ERROR_INVALID_MONITOR@ 0000000180005ca8     libattach009Agent00.obj
 0002:00000cc8       ??_C@_0BO@PPEDAJGL@JVMTI_ERROR_NOT_MONITOR_OWNER@ 0000000180005cc8     libattach009Agent00.obj
 0002:00000ce8       ??_C@_0BG@FCAIPEID@JVMTI_ERROR_INTERRUPT@ 0000000180005ce8     libattach009Agent00.obj
 0002:00000d00       ??_C@_0CB@EGDBNKOI@JVMTI_ERROR_INVALID_CLASS_FORMA@ 0000000180005d00     libattach009Agent00.obj
 0002:00000d28       ??_C@_0CG@DGKOGIAL@JVMTI_ERROR_CIRCULAR_CLASS_DEFI@ 0000000180005d28     libattach009Agent00.obj
 0002:00000d50       ??_C@_0BP@ICEALPKC@JVMTI_ERROR_FAILS_VERIFICATION@ 0000000180005d50     libattach009Agent00.obj
 0002:00000d70       ??_C@_0DC@JDACLMIO@JVMTI_ERROR_UNSUPPORTED_REDEFIN@ 0000000180005d70     libattach009Agent00.obj
 0002:00000da8       ??_C@_0DE@GKDKNOMJ@JVMTI_ERROR_UNSUPPORTED_REDEFIN@ 0000000180005da8     libattach009Agent00.obj
 0002:00000de0       ??_C@_0BO@LAFKIOG@JVMTI_ERROR_INVALID_TYPESTATE@ 0000000180005de0     libattach009Agent00.obj
 0002:00000e00       ??_C@_0DH@INDGCLLB@JVMTI_ERROR_UNSUPPORTED_REDEFIN@ 0000000180005e00     libattach009Agent00.obj
 0002:00000e38       ??_C@_0DE@NHEOMMGI@JVMTI_ERROR_UNSUPPORTED_REDEFIN@ 0000000180005e38     libattach009Agent00.obj
 0002:00000e70       ??_C@_0CA@EKPNJOEP@JVMTI_ERROR_UNSUPPORTED_VERSION@ 0000000180005e70     libattach009Agent00.obj
 0002:00000e90       ??_C@_0BN@OFFMAHHL@JVMTI_ERROR_NAMES_DONT_MATCH@ 0000000180005e90     libattach009Agent00.obj
 0002:00000eb0       ??_C@_0DN@HHBBLAKE@JVMTI_ERROR_UNSUPPORTED_REDEFIN@ 0000000180005eb0     libattach009Agent00.obj
 0002:00000ef0       ??_C@_0DO@HMBGBGNA@JVMTI_ERROR_UNSUPPORTED_REDEFIN@ 0000000180005ef0     libattach009Agent00.obj
 0002:00000f30       ??_C@_0BP@PBECGKHJ@JVMTI_ERROR_UNMODIFIABLE_CLASS@ 0000000180005f30     libattach009Agent00.obj
 0002:00000f50       ??_C@_0BK@CANILEHF@JVMTI_ERROR_NOT_AVAILABLE@ 0000000180005f50     libattach009Agent00.obj
 0002:00000f70       ??_C@_0CE@INJKMEFK@JVMTI_ERROR_MUST_POSSESS_CAPABI@ 0000000180005f70     libattach009Agent00.obj
 0002:00000f98       ??_C@_0BJ@LBFPFPDM@JVMTI_ERROR_NULL_POINTER@ 0000000180005f98     libattach009Agent00.obj
 0002:00000fb8       ??_C@_0BP@CHJPNNEM@JVMTI_ERROR_ABSENT_INFORMATION@ 0000000180005fb8     libattach009Agent00.obj
 0002:00000fd8       ??_C@_0BP@OMFMNLC@JVMTI_ERROR_INVALID_EVENT_TYPE@ 0000000180005fd8     libattach009Agent00.obj
 0002:00000ff8       ??_C@_0BN@BIBNPHHO@JVMTI_ERROR_ILLEGAL_ARGUMENT@ 0000000180005ff8     libattach009Agent00.obj
 0002:00001018       ??_C@_0BK@KKNDHDCE@JVMTI_ERROR_NATIVE_METHOD@ 0000000180006018     libattach009Agent00.obj
 0002:00001038       ??_C@_0BK@PMKCFHAE@JVMTI_ERROR_OUT_OF_MEMORY@ 0000000180006038     libattach009Agent00.obj
 0002:00001058       ??_C@_0BK@NNJBDMNB@JVMTI_ERROR_ACCESS_DENIED@ 0000000180006058     libattach009Agent00.obj
 0002:00001078       ??_C@_0BI@GHECLMNC@JVMTI_ERROR_WRONG_PHASE@ 0000000180006078     libattach009Agent00.obj
 0002:00001090       ??_C@_0BF@OLIHJOII@JVMTI_ERROR_INTERNAL@ 0000000180006090     libattach009Agent00.obj
 0002:000010a8       ??_C@_0BO@EOHGKJHI@JVMTI_ERROR_UNATTACHED_THREAD@ 00000001800060a8     libattach009Agent00.obj
 0002:000010c8       ??_C@_0CA@LKHFDACL@JVMTI_ERROR_INVALID_ENVIRONMENT@ 00000001800060c8     libattach009Agent00.obj
 0002:000010e8       ??_C@_0BA@MMFHLOKK@?$DMunknown?5error?$DO@ 00000001800060e8     libattach009Agent00.obj
 0002:000010f8       ??_C@_0CF@CBHOKDB@throwable?5?$DN?5jni?9?$DOExceptionOccur@ 00000001800060f8     libattach009Agent00.obj
 0002:00001120       ??_C@_03OFAPEBGM@?$CFs?6@  0000000180006120     libattach009Agent00.obj
 0002:00001128       ??_C@_0DM@LPIGEGNJ@s?2test?2hotspot?2jtreg?2vmTestbase@ 0000000180006128     libattach009Agent00.obj
 0002:00001168       ??_C@_0CC@NFCNPEPK@Exception?5in?5JNI?5call?5?$CIcleared?$CJ@ 0000000180006168     libattach009Agent00.obj
 0002:00001190       ??_C@_0BJ@IBAKFIKF@jni?9?$DOExceptionDescribe?$CI?$CJ@ 0000000180006190     libattach009Agent00.obj
 0002:000011b0       ??_C@_0BG@GGKALKMH@jni?9?$DOExceptionClear?$CI?$CJ@ 00000001800061b0     libattach009Agent00.obj
 0002:000011c8       ??_C@_0CF@JMGFGJLJ@?$CD?5?5?5verified?5JNI?5assertion?5is?5F@ 00000001800061c8     libattach009Agent00.obj
 0002:000011f0       ??_C@_0CB@MLNJNCLJ@?5?5jvmti?5error?3?5code?$DN?$CFd?0?5name?$DN?$CFs@ 00000001800061f0     libattach009Agent00.obj
 0002:00001218       ??_C@_0CD@OHBGDKMK@?$CD?5?5?5jvmti?5error?3?5code?$DN?$CFd?0?5name?$DN@ 0000000180006218     libattach009Agent00.obj
 0002:00001240       ??_C@_0CG@JNNCGPHB@?$CD?5?5?5error?5expected?3?5code?$DN?$CFd?0?5na@ 0000000180006240     libattach009Agent00.obj
 0002:00001270       ??_C@_0EB@IMGKPCGE@?$CIstr_obj?5?$DN?5jni?9?$DONewStringUTF?$CIco@ 0000000180006270     libattach009Agent00.obj
 0002:000012c0       ??_C@_0EA@HFOGGBCC@s?2test?2hotspot?2jtreg?2vmTestbase@ 00000001800062c0     libattach009Agent00.obj
 0002:00001300       ??_C@_05KKCIMGE@error@     0000000180006300     libattach009Agent00.obj
 0002:00001308       ??_C@_0CJ@JACLEAA@Test?5failed?5by?5setFailStatus?$CI?$CJ?4@ 0000000180006308     libattach009Agent00.obj
 0002:00001338       ??_C@_0BD@HGNAOMCP@agent_data_monitor@ 0000000180006338     libattach009Agent00.obj
 0002:00001350       ??_C@_0EB@OGCLGKLN@javaVM?9?$DOGetEnv?$CI?$CIvoid?5?$CK?$CK?$CJ?$CGjvmti_@ 0000000180006350     libattach009Agent00.obj
 0002:000013a0       ??_C@_0EA@PNBCDMOA@s?2test?2hotspot?2jtreg?2vmTestbase@ 00000001800063a0     libattach009Agent00.obj
 0002:000013e0       ??_C@_0CI@DDPIFBGM@init_agent_data?$CIjvmti_env?0?5?$CGage@ 00000001800063e0     libattach009Agent00.obj
 0002:00001408       ??_C@_0DI@ILAHDLMP@?$CI?$CKagentThreadProc?$CJ?$CIjvmti_env?0?5a@ 0000000180006408     libattach009Agent00.obj
 0002:00001440       ??_C@_0BD@KDBALNLB@JVMTI?5agent?5thread@ 0000000180006440     libattach009Agent00.obj
 0002:00001458       ??_C@_0BB@NOKBFPFO@java?1lang?1Thread@ 0000000180006458     libattach009Agent00.obj
 0002:0000146c       ??_C@_06FALKBLGB@?$DMinit?$DO@ 000000018000646c     libattach009Agent00.obj
 0002:00001480       ??_C@_0EB@IFJBFEKC@?$CIthreadClass?5?$DN?5jni_env?9?$DOFindCla@ 0000000180006480     libattach009Agent00.obj
 0002:000014d0       ??_C@_0GF@FGFIBKKL@?$CIthreadCtor?5?$DN?5jni_env?9?$DOGetMetho@ 00000001800064d0     libattach009Agent00.obj
 0002:00001538       ??_C@_0DN@NCPDJLOG@?$CIthreadName?5?$DN?5jni_env?9?$DONewStrin@ 0000000180006538     libattach009Agent00.obj
 0002:00001580       ??_C@_0FE@PFKODBGC@?$CIthreadObject?5?$DN?5jni_env?9?$DONewObj@ 0000000180006580     libattach009Agent00.obj
 0002:000015e0       ??_C@_0ED@HOBAHHJI@?$CIthreadGlobalRef?5?$DN?5jni_env?9?$DONew@ 00000001800065e0     libattach009Agent00.obj
 0002:00001630       ??_C@_0FN@HNJJAHFC@jvmti_env?9?$DORunAgentThread?$CIagent@ 0000000180006630     libattach009Agent00.obj
 0002:00001690       ??_C@_0EA@MOJDNKDF@Debuggee?5status?5sync?5aborted?5be@ 0000000180006690     libattach009Agent00.obj
 0002:000016d0       ??_C@_0EA@EEOEJAEN@status?5?$DN?5syncDebuggeeStatus?$CIjni@ 00000001800066d0     libattach009Agent00.obj
 0002:00001710       ??_C@_0BL@JBCFNBMB@nsk_jvmti_resetAgentData?$CI?$CJ@ 0000000180006710     libattach009Agent00.obj
 0002:00001730       ??_C@_0EL@LPBEELIP@s?2test?2hotspot?2jtreg?2vmTestbase@ 0000000180006730     libattach009Agent00.obj
 0002:00001780       ??_C@_0CK@JDAMFDMJ@jvmti?9?$DOSetTag?$CIo?0?5tag?$CJ?5?$DN?$DN?5JVMTI_@ 0000000180006780     libattach009Agent00.obj
 0002:000017b0       ??_C@_0CC@DAMNHKNI@Can?8t?5set?5tag?5?$CFli?5for?5object?5?$CFl@ 00000001800067b0     libattach009Agent00.obj
 0002:000017d8       ??_C@_0DL@HAJPNKEF@jvmti?9?$DOGetObjectHashCode?$CIo?0?5?$CGha@ 00000001800067d8     libattach009Agent00.obj
 0002:00001818       ??_C@_0BL@JFPIEOBF@Can?8t?5get?5hash?5object?5?$CFlx?6@ 0000000180006818     libattach009Agent00.obj
 0002:00001838       ??_C@_0BG@DICPHBKN@setTag?3?5?$CF08x?5?$DM?9?5?$CF?53li@ 0000000180006838     libattach009Agent00.obj
 0002:00001850       ??_C@_0DH@FCEEBDMJ@?$CIs?5?$DN?5jni?9?$DOGetStringUTFChars?$CIsIn@ 0000000180006850     libattach009Agent00.obj
 0002:00001888       ??_C@_0BJ@OKKGHDCN@Can?8t?5get?5string?5at?5?$CF?$CDp?6@ 0000000180006888     libattach009Agent00.obj
 0002:000018a8       ??_C@_0BP@EKFLGGFJ@Can?8t?5get?5string?5at?5?$CF?$CDp?3?5null?6@ 00000001800068a8     libattach009Agent00.obj
 0002:000018c8       ??_C@_06ICODBHCL@?5?1?1?5?$CFs@ 00000001800068c8     libattach009Agent00.obj
 0002:000018d0       ??_C@_0DB@KGFPLEGO@?$CIr?5?$DN?5jvmti?9?$DOGetTag?$CIo?0?5?$CGtag?$CJ?$CJ?5?$DN?$DN@ 00000001800068d0     libattach009Agent00.obj
 0002:00001908       ??_C@_0CO@PDAGBCGJ@Can?8t?5GetTag?5for?5object?5?$CFlx?4?5Re@ 0000000180006908     libattach009Agent00.obj
 0002:00001938       ??_C@_0CH@HPEODOHC@TEST_BUG?3?5Max?4?5number?5of?5refs?5r@ 0000000180006938     libattach009Agent00.obj
 0002:00001960       ??_C@_0DI@PHFCABIM@?$CIr?5?$DN?5jvmti?9?$DOGetTag?$CIfrom?0?5?$CGtagFr@ 0000000180006960     libattach009Agent00.obj
 0002:00001998       ??_C@_0DI@MDEGFNKD@TEST_BUG?3?5Can?8t?5GetTag?5for?5obje@ 0000000180006998     libattach009Agent00.obj
 0002:000019d0       ??_C@_0DE@MLELJAHM@?$CIr?5?$DN?5jvmti?9?$DOGetTag?$CIto?0?5?$CGtagTo?$CJ?$CJ@ 00000001800069d0     libattach009Agent00.obj
 0002:00001a08       ??_C@_0CF@NBAMCKHO@Unexpected?5exception?5after?5JNI?5@ 0000000180006a08     libattach009Agent00.obj
 0002:00001a30       ??_C@_0DG@ECLJIGOO@s?2test?2hotspot?2jtreg?2vmTestbase@ 0000000180006a30     libattach009Agent00.obj
 0002:00001a70       ??_C@_0EK@CABJMPML@WARNING?3?5some?5error?5happened?5in@ 0000000180006a70     libattach009Agent00.obj
 0002:00001ac0       ??_C@_0CN@EDIMGGCE@options?5were?5not?5passed?5to?5the?5@ 0000000180006ac0     libattach009Agent00.obj
 0002:00001af0       ??_C@_0BO@HIBNDEOE@Invalid?5options?5format?3?5?8?$CFs?8?6@ 0000000180006af0     libattach009Agent00.obj
 0002:00001b10       ??_C@_0BG@BCGDCLLA@Option?5?8?$CFs?8?5is?5empty?6@ 0000000180006b10     libattach009Agent00.obj
 0002:00001b30       ??_C@_0EI@CFFDGDKG@WARNING?3?5not?5all?5options?5were?5p@ 0000000180006b30     libattach009Agent00.obj
 0002:00001b80       ??_C@_0EN@LHKBBCDP@?$CIoptions?5?$DN?5?$CIOptions?$CK?$CJ?5nsk_aod_c@ 0000000180006b80     libattach009Agent00.obj
 0002:00001bd0       ??_C@_0DM@MFFOLIAC@nsk_aod_optionSpecified?$CIoptions@ 0000000180006bd0     libattach009Agent00.obj
 0002:00001c10       ??_C@_0L@DALKGIIP@?9agentName@ 0000000180006c10     libattach009Agent00.obj
 0002:00001c20       ??_C@_0BN@PFMBIOBG@Agent?5name?5wasn?8t?5specified?6@ 0000000180006c20     libattach009Agent00.obj
 0002:00001c40       ??_C@_08FBJJFDKJ@?9verbose@ 0000000180006c40     libattach009Agent00.obj
 0002:00001c4c       ??_C@_05LAPONLG@false@     0000000180006c4c     libattach009Agent00.obj
 0002:00001c58       ??_C@_0BD@FMBAOLJK@options?5?$CB?$DN?5nullptr@ 0000000180006c58     libattach009Agent00.obj
 0002:00001c70       ??_C@_0O@BPHJJCEJ@Options?5null?6@ 0000000180006c70     libattach009Agent00.obj
 0002:00001c80       ??_C@_0BL@NJPPLGIO@Option?5?8?$CFs?8?5isn?8t?5defined?6@ 0000000180006c80     libattach009Agent00.obj
 0002:00001ca0       ??_C@_0BE@DNNCOIDF@Agent?5?$CFs?5is?5loaded?6@ 0000000180006ca0     libattach009Agent00.obj
 0002:00001cc0       ??_C@_0EJ@NDOPGKMK@?$CIlocalTargetAppClass?5?$DN?5jni?9?$DOFin@ 0000000180006cc0     libattach009Agent00.obj
 0002:00001d10       ??_C@_0EO@HKMHFBAF@?$CItargetAppClass?5?$DN?5?$CIjclass?$CJ?5jni?9@ 0000000180006d10     libattach009Agent00.obj
 0002:00001d60       ??_C@_0IB@FFOAAHNN@?$CIagentLoadedMethod?5?$DN?5jni?9?$DOGetSt@ 0000000180006d60     libattach009Agent00.obj
 0002:00001de8       ??_C@_0DM@HLLJGLFL@?$CIagentNameString?5?$DN?5jni?9?$DONewStri@ 0000000180006de8     libattach009Agent00.obj
 0002:00001e30       ??_C@_0FP@EEAOJLDE@?$CFs?3?5TEST?5LOGIC?5ERROR?3?5method?5?8a@ 0000000180006e30     libattach009Agent00.obj
 0002:00001e90       ??_C@_0II@KPBFKHFM@Status?5of?5agent?5?8?$CFs?8?5is?5?8passed@ 0000000180006e90     libattach009Agent00.obj
 0002:00001f18       ??_C@_0CB@ECJEOOED@Agent?5?$CFs?5finished?5?$CIsuccess?3?5?$CFd?$CJ@ 0000000180006f18     libattach009Agent00.obj
 0002:00001f40       ??_C@_0IH@FIFEINGM@?$CIagentFinishedMethod?5?$DN?5jni?9?$DOGet@ 0000000180006f40     libattach009Agent00.obj
 0002:00001fc8       ??_C@_0P@POOJKNDK@jni?5?$CB?$DN?5nullptr@ 0000000180006fc8     libattach009Agent00.obj
 0002:00001fd8       ??_C@_0DP@GNGOCDGE@jvmti?9?$DOSetEventNotificationMode@ 0000000180006fd8     libattach009Agent00.obj
 0002:00002020       ??_C@_0EC@LNOIGMCL@s?2test?2hotspot?2jtreg?2vmTestbase@ 0000000180007020     libattach009Agent00.obj
 0002:00002068       ??_C@_0BH@DFACKHAD@jvmti?9?$DODeallocate?$CImem?$CJ@ 0000000180007068     libattach009Agent00.obj
 0002:00002080       ??_C@_0BD@DPLLDHNC@Deallocate?5failed?6@ 0000000180007080     libattach009Agent00.obj
 0002:00002098       ??_C@_0DF@HIDMGHGJ@jvmti?9?$DOGetClassSignature?$CIklass?0@ 0000000180007098     libattach009Agent00.obj
 0002:000020d0       ??_C@_0BK@EEHGBOLL@Failed?5to?5get?5class?5name?6@ 00000001800070d0     libattach009Agent00.obj
 0002:000020f0       ??_C@_0CE@LGKCCDOO@jvmti?9?$DOGetThreadInfo?$CIthread?0?5?$CGi@ 00000001800070f0     libattach009Agent00.obj
 0002:00002118       ??_C@_0BL@LNEBMKFE@Failed?5to?5get?5thread?5info?6@ 0000000180007118     libattach009Agent00.obj
 0002:00002138       ??_C@_0CG@KIBPLOAK@Class?5?8?$CFs?8?5was?5loaded?5by?5thread@ 0000000180007138     libattach009Agent00.obj
 0002:00002160       ??_C@_0FI@LIKDJLNF@s?2test?2hotspot?2jtreg?2vmTestbase@ 0000000180007160     libattach009Agent00.obj
 0002:000021b8       ??_C@_0DG@BEPHJMCC@Lnsk?1jvmti?1AttachOnDemand?1attac@ 00000001800071b8     libattach009Agent00.obj
 0002:000021f0       ??_C@_0FA@JEJOBGFM@jvmti?9?$DOSetEventNotificationMode@ 00000001800071f0     libattach009Agent00.obj
 0002:00002240       ??_C@_0BK@NDPADEAB@Failed?5to?5disable?5events?6@ 0000000180007240     libattach009Agent00.obj
 0002:00002260       ??_C@_0EO@ENGNCFCK@jvmti?9?$DOSetEventNotificationMode@ 0000000180007260     libattach009Agent00.obj
 0002:000022b0       ??_C@_0CJ@JEMLPLPL@Failed?5to?5enable?5events?5for?5thr@ 00000001800072b0     libattach009Agent00.obj
 0002:000022e0       ??_C@_0DC@IJJKLNCD@ClassLoad?5events?5are?5enabled?5on@ 00000001800072e0     libattach009Agent00.obj
 0002:00002318       ??_C@_0DL@DBGJPCBB@ClassLoad?5event?5was?5erroneously@ 0000000180007318     libattach009Agent00.obj
 0002:00002358       ??_C@_0DF@EBFJFIIK@Lnsk?1jvmti?1AttachOnDemand?1attac@ 0000000180007358     libattach009Agent00.obj
 0002:00002390       ??_C@_0BB@CGPOECH@jvmti?5?$CB?$DN?5nullptr@ 0000000180007390     libattach009Agent00.obj
 0002:000023b0       ??_C@_0EC@ODFGFOAJ@jvmti?9?$DOSetEventCallbacks?$CI?$CGevent@ 00000001800073b0     libattach009Agent00.obj
 0002:00002400       ??_C@_0EP@DMHOEJKK@jvmti?9?$DOSetEventNotificationMode@ 0000000180007400     libattach009Agent00.obj
 0002:00002450       ??_C@_0BN@GGABIMJA@?$CFs?3?5initialization?5was?5done?6@ 0000000180007450     libattach009Agent00.obj
 0002:00002470       ??_C@_0CE@PACICCLF@nsk_aod_agentLoaded?$CIjni?0?5agentN@ 0000000180007470     libattach009Agent00.obj
 0002:000024b0       ??_C@_1EC@JIJBPKFM@?$AAa?$AAp?$AAi?$AA?9?$AAm?$AAs?$AA?9?$AAw?$AAi?$AAn?$AA?9?$AAc?$AAo?$AAr?$AAe@ 00000001800074b0     MSVCRT:thread_safe_statics.obj
 0002:000024f8       ??_C@_1BK@MGMFAEKH@?$AAk?$AAe?$AAr?$AAn?$AAe?$AAl?$AA3?$AA2?$AA?4?$AAd?$AAl?$AAl@ 00000001800074f8     MSVCRT:thread_safe_statics.obj
 0002:00002518       ??_C@_0BJ@JEBJOJFJ@SleepConditionVariableCS@ 0000000180007518     MSVCRT:thread_safe_statics.obj
 0002:00002538       ??_C@_0BJ@PGPPEPCC@WakeAllConditionVariable@ 0000000180007538     MSVCRT:thread_safe_statics.obj
 0002:00002558       _pDefaultRawDllMain        0000000180007558     MSVCRT:dll_dllmain.obj
 0002:00002558       _pRawDllMain               0000000180007558     MSVCRT:dll_dllmain.obj
 0002:00002560       __xmm@ffffffffffffffffffffffffffffffff 0000000180007560     MSVCRT:utility.obj
 0002:00002570       _load_config_used          0000000180007570     MSVCRT:loadcfg.obj
 0002:00002780       _tls_used                  0000000180007780     MSVCRT:tlssup.obj
 0002:000027a8       __volatile_metadata        00000001800077a8     <linker-defined>
 0002:00002b80       __rtc_iaa                  0000000180007b80     MSVCRT:initsect.obj
 0002:00002b88       __rtc_izz                  0000000180007b88     MSVCRT:initsect.obj
 0002:00002b90       __rtc_taa                  0000000180007b90     MSVCRT:initsect.obj
 0002:00002b98       __rtc_tzz                  0000000180007b98     MSVCRT:initsect.obj
 0002:00002ba0       _tls_start                 0000000180007ba0     MSVCRT:tlssup.obj
 0002:00002ba4       _Init_thread_epoch         0000000180007ba4     MSVCRT:thread_safe_statics.obj
 0002:00002ba8       _tls_end                   0000000180007ba8     MSVCRT:tlssup.obj
 0002:000032c4       __IMPORT_DESCRIPTOR_KERNEL32 00000001800082c4     kernel32:KERNEL32.dll
 0002:000032d8       __IMPORT_DESCRIPTOR_VCRUNTIME140 00000001800082d8     vcruntime:VCRUNTIME140.dll
 0002:000032ec       __IMPORT_DESCRIPTOR_api-ms-win-crt-heap-l1-1-0 00000001800082ec     ucrt:api-ms-win-crt-heap-l1-1-0.dll
 0002:00003300       __IMPORT_DESCRIPTOR_api-ms-win-crt-runtime-l1-1-0 0000000180008300     ucrt:api-ms-win-crt-runtime-l1-1-0.dll
 0002:00003314       __IMPORT_DESCRIPTOR_api-ms-win-crt-stdio-l1-1-0 0000000180008314     ucrt:api-ms-win-crt-stdio-l1-1-0.dll
 0002:00003328       __IMPORT_DESCRIPTOR_api-ms-win-crt-string-l1-1-0 0000000180008328     ucrt:api-ms-win-crt-string-l1-1-0.dll
 0002:0000333c       __NULL_IMPORT_DESCRIPTOR   000000018000833c     kernel32:KERNEL32.dll
 0003:0000005c       _Init_global_epoch         000000018000905c     MSVCRT:thread_safe_statics.obj
 0003:00000060       __security_cookie          0000000180009060     MSVCRT:gs_cookie.obj
 0003:00000068       __security_cookie_complement 0000000180009068     MSVCRT:gs_cookie.obj
 0003:00000070       __scrt_native_dllmain_reason 0000000180009070     MSVCRT:utility.obj
 0003:00000078       __isa_available            0000000180009078     MSVCRT:cpu_disp.obj
 0003:0000007c       __isa_enabled              000000018000907c     MSVCRT:cpu_disp.obj
 0003:00000080       __memset_fast_string_threshold 0000000180009080     MSVCRT:cpu_disp.obj
 0003:00000088       __memset_nt_threshold      0000000180009088     MSVCRT:cpu_disp.obj
 0003:00000090       __scrt_ucrt_dll_is_in_use  0000000180009090     MSVCRT:ucrt_stubs.obj
 0003:000000a0       g_wrongHeapCallbacks       00000001800090a0     libattach009Agent00.obj
 0003:00000120       g_szTagInfo                0000000180009120     libattach009Agent00.obj
 0003:00002060       g_tagFlags                 000000018000b060     libattach009Agent00.obj
 0003:00002448       g_refsToVerifyCnt          000000018000b448     libattach009Agent00.obj
 0003:0000244c       g_fakeUserData             000000018000b44c     libattach009Agent00.obj
 0003:00002450       g_tagVisitCount            000000018000b450     libattach009Agent00.obj
 0003:000033f0       g_refsToVerify             000000018000c3f0     libattach009Agent00.obj
 0003:0001aaf0       g_userDataError            0000000180023af0     libattach009Agent00.obj
 0003:0001ab00       multiagentsOptions         0000000180023b00     libattach009Agent00.obj
 0003:0001ad68       ?_OptionsStorage@?1??__local_stdio_printf_options@@9@4_KA 0000000180023d68     libattach009Agent00.obj
 0003:0001b728       _tls_index                 0000000180024728     MSVCRT:tlssup.obj
 0003:0001b730       __scrt_current_native_startup_state 0000000180024730     MSVCRT:utility.obj
 0003:0001b738       __scrt_native_startup_lock 0000000180024738     MSVCRT:utility.obj
 0003:0001b778       __scrt_debugger_hook_flag  0000000180024778     MSVCRT:utility_desktop.obj
 0003:0001b780       ?__type_info_root_node@@3U__type_info_node@@A 0000000180024780     MSVCRT:tncleanup.obj
 0003:0001b790       ?_OptionsStorage@?1??__local_stdio_scanf_options@@9@4_KA 0000000180024790     MSVCRT:default_local_stdio_options.obj
 0003:0001b798       __favor                    0000000180024798     MSVCRT:cpu_disp.obj
 0003:0001b7a0       __dyn_tls_init_callback    00000001800247a0     <common>

 entry point at        0001:000033d0

 Static symbols

 0000:fffd9000       .debug$S                   0000000180000000     attach009Agent00.exp
 0000:fffd9000       .debug$S                   0000000180000000     vcruntime:VCRUNTIME140.dll
 0000:fffd9000       .debug$S                   0000000180000000     vcruntime:VCRUNTIME140.dll
 0000:fffd9000       .debug$S                   0000000180000000     vcruntime:VCRUNTIME140.dll
 0000:fffd9000       .debug$S                   0000000180000000     vcruntime:VCRUNTIME140.dll
 0000:fffd9000       .debug$S                   0000000180000000     vcruntime:VCRUNTIME140.dll
 0000:fffd9000       .debug$S                   0000000180000000     vcruntime:VCRUNTIME140.dll
 0000:fffd9000       .debug$S                   0000000180000000     vcruntime:VCRUNTIME140.dll
 0000:fffd9000       .debug$S                   0000000180000000     ucrt:api-ms-win-crt-convert-l1-1-0.dll
 0002:ffffb000       .idata$6                   0000000180000000     ucrt:api-ms-win-crt-convert-l1-1-0.dll
 0000:fffd9000       .debug$S                   0000000180000000     ucrt:api-ms-win-crt-heap-l1-1-0.dll
 0000:fffd9000       .debug$S                   0000000180000000     ucrt:api-ms-win-crt-heap-l1-1-0.dll
 0000:fffd9000       .debug$S                   0000000180000000     ucrt:api-ms-win-crt-heap-l1-1-0.dll
 0000:fffd9000       .debug$S                   0000000180000000     ucrt:api-ms-win-crt-heap-l1-1-0.dll
 0000:fffd9000       .debug$S                   0000000180000000     ucrt:api-ms-win-crt-runtime-l1-1-0.dll
 0000:fffd9000       .debug$S                   0000000180000000     ucrt:api-ms-win-crt-runtime-l1-1-0.dll
 0000:fffd9000       .debug$S                   0000000180000000     ucrt:api-ms-win-crt-runtime-l1-1-0.dll
 0000:fffd9000       .debug$S                   0000000180000000     ucrt:api-ms-win-crt-runtime-l1-1-0.dll
 0000:fffd9000       .debug$S                   0000000180000000     ucrt:api-ms-win-crt-runtime-l1-1-0.dll
 0000:fffd9000       .debug$S                   0000000180000000     ucrt:api-ms-win-crt-runtime-l1-1-0.dll
 0000:fffd9000       .debug$S                   0000000180000000     ucrt:api-ms-win-crt-runtime-l1-1-0.dll
 0000:fffd9000       .debug$S                   0000000180000000     ucrt:api-ms-win-crt-runtime-l1-1-0.dll
 0000:fffd9000       .debug$S                   0000000180000000     ucrt:api-ms-win-crt-runtime-l1-1-0.dll
 0000:fffd9000       .debug$S                   0000000180000000     ucrt:api-ms-win-crt-runtime-l1-1-0.dll
 0000:fffd9000       .debug$S                   0000000180000000     ucrt:api-ms-win-crt-runtime-l1-1-0.dll
 0000:fffd9000       .debug$S                   0000000180000000     ucrt:api-ms-win-crt-runtime-l1-1-0.dll
 0000:fffd9000       .debug$S                   0000000180000000     ucrt:api-ms-win-crt-runtime-l1-1-0.dll
 0000:fffd9000       .debug$S                   0000000180000000     ucrt:api-ms-win-crt-runtime-l1-1-0.dll
 0000:fffd9000       .debug$S                   0000000180000000     ucrt:api-ms-win-crt-runtime-l1-1-0.dll
 0000:fffd9000       .debug$S                   0000000180000000     ucrt:api-ms-win-crt-runtime-l1-1-0.dll
 0000:fffd9000       .debug$S                   0000000180000000     ucrt:api-ms-win-crt-stdio-l1-1-0.dll
 0000:fffd9000       .debug$S                   0000000180000000     ucrt:api-ms-win-crt-stdio-l1-1-0.dll
 0000:fffd9000       .debug$S                   0000000180000000     ucrt:api-ms-win-crt-stdio-l1-1-0.dll
 0000:fffd9000       .debug$S                   0000000180000000     ucrt:api-ms-win-crt-stdio-l1-1-0.dll
 0000:fffd9000       .debug$S                   0000000180000000     ucrt:api-ms-win-crt-stdio-l1-1-0.dll
 0000:fffd9000       .debug$S                   0000000180000000     ucrt:api-ms-win-crt-stdio-l1-1-0.dll
 0000:fffd9000       .debug$S                   0000000180000000     ucrt:api-ms-win-crt-stdio-l1-1-0.dll
 0000:fffd9000       .debug$S                   0000000180000000     ucrt:api-ms-win-crt-stdio-l1-1-0.dll
 0000:fffd9000       .debug$S                   0000000180000000     ucrt:api-ms-win-crt-stdio-l1-1-0.dll
 0000:fffd9000       .debug$S                   0000000180000000     ucrt:api-ms-win-crt-stdio-l1-1-0.dll
 0000:fffd9000       .debug$S                   0000000180000000     ucrt:api-ms-win-crt-string-l1-1-0.dll
 0000:fffd9000       .debug$S                   0000000180000000     ucrt:api-ms-win-crt-string-l1-1-0.dll
 0000:fffd9000       .debug$S                   0000000180000000     ucrt:api-ms-win-crt-string-l1-1-0.dll
 0000:fffd9000       .debug$S                   0000000180000000     ucrt:api-ms-win-crt-string-l1-1-0.dll
 0000:fffd9000       .debug$S                   0000000180000000     ucrt:api-ms-win-crt-string-l1-1-0.dll
 0000:fffd9000       .debug$S                   0000000180000000     ucrt:api-ms-win-crt-string-l1-1-0.dll
 0000:fffd9000       .debug$S                   0000000180000000     ucrt:api-ms-win-crt-string-l1-1-0.dll
 0000:fffd9000       .debug$S                   0000000180000000     ucrt:api-ms-win-crt-string-l1-1-0.dll
 0000:fffd9000       .debug$S                   0000000180000000     ucrt:api-ms-win-crt-string-l1-1-0.dll
 0000:fffd9000       .debug$S                   0000000180000000     kernel32:KERNEL32.dll
 0000:fffd9000       .debug$S                   0000000180000000     kernel32:KERNEL32.dll
 0000:fffd9000       .debug$S                   0000000180000000     kernel32:KERNEL32.dll
 0000:fffd9000       .debug$S                   0000000180000000     kernel32:KERNEL32.dll
 0000:fffd9000       .debug$S                   0000000180000000     kernel32:KERNEL32.dll
 0000:fffd9000       .debug$S                   0000000180000000     kernel32:KERNEL32.dll
 0000:fffd9000       .debug$S                   0000000180000000     kernel32:KERNEL32.dll
 0000:fffd9000       .debug$S                   0000000180000000     kernel32:KERNEL32.dll
 0000:fffd9000       .debug$S                   0000000180000000     kernel32:KERNEL32.dll
 0000:fffd9000       .debug$S                   0000000180000000     kernel32:KERNEL32.dll
 0000:fffd9000       .debug$S                   0000000180000000     kernel32:KERNEL32.dll
 0000:fffd9000       .debug$S                   0000000180000000     kernel32:KERNEL32.dll
 0000:fffd9000       .debug$S                   0000000180000000     kernel32:KERNEL32.dll
 0000:fffd9000       .debug$S                   0000000180000000     kernel32:KERNEL32.dll
 0000:fffd9000       .debug$S                   0000000180000000     kernel32:KERNEL32.dll
 0000:fffd9000       .debug$S                   0000000180000000     kernel32:KERNEL32.dll
 0000:fffd9000       .debug$S                   0000000180000000     kernel32:KERNEL32.dll
 0000:fffd9000       .debug$S                   0000000180000000     kernel32:KERNEL32.dll
 0000:fffd9000       .debug$S                   0000000180000000     kernel32:KERNEL32.dll
 0000:fffd9000       .debug$S                   0000000180000000     kernel32:KERNEL32.dll
 0000:fffd9000       .debug$S                   0000000180000000     kernel32:KERNEL32.dll
 0000:fffd9000       .debug$S                   0000000180000000     kernel32:KERNEL32.dll
 0000:fffd9000       .debug$S                   0000000180000000     kernel32:KERNEL32.dll
 0000:fffd9000       .debug$S                   0000000180000000     kernel32:KERNEL32.dll
 0000:fffd9000       .debug$S                   0000000180000000     kernel32:KERNEL32.dll
 0000:fffd9000       .debug$S                   0000000180000000     kernel32:KERNEL32.dll
 0000:fffd9000       .debug$S                   0000000180000000     kernel32:KERNEL32.dll
 0000:fffd9000       .debug$S                   0000000180000000     kernel32:KERNEL32.dll
 0001:00000f1c       addRefToVerify             0000000180001f1c f   libattach009Agent00.obj
 0001:00000f88       agentThreadWrapper         0000000180001f88 f   libattach009Agent00.obj
 0001:000013e8       file_basename              00000001800023e8 f   libattach009Agent00.obj
 0001:000018d0       nsk_aod_checkJNIException  00000001800028d0 f   libattach009Agent00.obj
 0001:000028ac       startAgentThreadWrapper    00000001800038ac f   libattach009Agent00.obj
 0001:00002bec       syncDebuggeeStatus         0000000180003bec f   libattach009Agent00.obj
 0001:00002e8c       capture_previous_context   0000000180003e8c f   MSVCRT:gs_report.obj
 0001:00002f00       ?__scrt_initialize_thread_safe_statics@@YAHXZ 0000000180003f00 f   MSVCRT:thread_safe_statics.obj
 0001:00002fd0       ?__scrt_uninitialize_thread_safe_statics@@YAXXZ 0000000180003fd0 f   MSVCRT:thread_safe_statics.obj
 0001:00003080       $$000000                   0000000180004080     MSVCRT:amdsecgs.obj
 0001:000030b0       ?dllmain_crt_dispatch@@YAHQEAUHINSTANCE__@@KQEAX@Z 00000001800040b0 f   MSVCRT:dll_dllmain.obj
 0001:00003100       ?dllmain_crt_process_attach@@YAHQEAUHINSTANCE__@@QEAX@Z 0000000180004100 f   MSVCRT:dll_dllmain.obj
 0001:00003218       ?dllmain_crt_process_detach@@YAH_N@Z 0000000180004218 f   MSVCRT:dll_dllmain.obj
 0001:0000329c       ?dllmain_dispatch@@YAHQEAUHINSTANCE__@@KQEAX@Z 000000018000429c f   MSVCRT:dll_dllmain.obj
 0001:00003cc0       $$000000                   0000000180004cc0     MSVCRT:guard_dispatch.obj
 0001:00003ce0       $$000000                   0000000180004ce0     MSVCRT:guard_xfg_dispatch.obj
 0001:00003cf6       ?fin$0@?0??dllmain_crt_process_attach@@YAHQEAUHINSTANCE__@@QEAX@Z@4HA 0000000180004cf6 f   MSVCRT:dll_dllmain.obj
 0001:00003d0d       ?fin$0@?0??dllmain_crt_process_detach@@YAH_N@Z@4HA 0000000180004d0d f   MSVCRT:dll_dllmain.obj
 0001:00003d26       ?fin$1@?0??dllmain_crt_process_detach@@YAH_N@Z@4HA 0000000180004d26 f   MSVCRT:dll_dllmain.obj
 0001:00003d3a       ?filt$0@?0??dllmain_dispatch@@YAHQEAUHINSTANCE__@@KQEAX@Z@4HA 0000000180004d3a f   MSVCRT:dll_dllmain.obj
 0001:00003d70       __scrt_is_nonwritable_in_current_image$filt$0 0000000180004d70 f   MSVCRT:utility.obj
 0002:00000208       ?__scrt_initialize_tss_var@@3P6AHXZEA 0000000180005208     MSVCRT:thread_safe_statics.obj
 0002:00000350       ?opcLengths@@3QBEB         0000000180005350     libattach009Agent00.obj
 0002:00002498       GS_ExceptionPointers       0000000180007498     MSVCRT:gs_report.obj
 0002:00002bb0       $unwind$fprintf            0000000180007bb0     libattach009Agent00.obj
 0002:00002bbc       $unwind$printf             0000000180007bbc     libattach009Agent00.obj
 0002:00002bc8       $unwind$?CallStaticVoidMethod@JNIEnv_@@QEAAXPEAV_jclass@@PEAU_jmethodID@@ZZ 0000000180007bc8     libattach009Agent00.obj
 0002:00002bc8       $unwind$?NewObject@JNIEnv_@@QEAAPEAV_jobject@@PEAV_jclass@@PEAU_jmethodID@@ZZ 0000000180007bc8     libattach009Agent00.obj
 0002:00002bc8       $unwind$nsk_lcomplain      0000000180007bc8     libattach009Agent00.obj
 0002:00002bc8       $unwind$nsk_ldisplay       0000000180007bc8     libattach009Agent00.obj
 0002:00002bd0       $unwind$nsk_lvdisplay      0000000180007bd0     libattach009Agent00.obj
 0002:00002bd0       $unwind$_RTC_Initialize    0000000180007bd0     MSVCRT:initsect.obj
 0002:00002bd0       $unwind$_RTC_Terminate     0000000180007bd0     MSVCRT:initsect.obj
 0002:00002bd0       $unwind$?__scrt_initialize_thread_safe_statics@@YAHXZ 0000000180007bd0     MSVCRT:thread_safe_statics.obj
 0002:00002bdc       $unwind$nsk_lvcomplain     0000000180007bdc     libattach009Agent00.obj
 0002:00002bf4       $unwind$nsk_ltrace         0000000180007bf4     libattach009Agent00.obj
 0002:00002bf4       $unwind$__report_gsfailure 0000000180007bf4     MSVCRT:gs_report.obj
 0002:00002bfc       $unwind$nsk_aod_checkJNIException 0000000180007bfc     libattach009Agent00.obj
 0002:00002bfc       $unwind$nsk_lvtrace        0000000180007bfc     libattach009Agent00.obj
 0002:00002bfc       $unwind$__raise_securityfailure 0000000180007bfc     MSVCRT:gs_report.obj
 0002:00002bfc       $unwind$__scrt_initialize_crt 0000000180007bfc     MSVCRT:utility.obj
 0002:00002bfc       $unwind$__scrt_initialize_onexit_tables 0000000180007bfc     MSVCRT:utility.obj
 0002:00002bfc       $unwind$__scrt_release_startup_lock 0000000180007bfc     MSVCRT:utility.obj
 0002:00002bfc       $unwind$__scrt_uninitialize_crt 0000000180007bfc     MSVCRT:utility.obj
 0002:00002bfc       $unwind$_onexit            0000000180007bfc     MSVCRT:utility.obj
 0002:00002c04       $unwind$nsk_lverify        0000000180007c04     libattach009Agent00.obj
 0002:00002c14       $unwind$nsk_vprintf        0000000180007c14     libattach009Agent00.obj
 0002:00002c24       $unwind$nsk_printf         0000000180007c24     libattach009Agent00.obj
 0002:00002c2c       $unwind$Agent_OnAttach     0000000180007c2c     libattach009Agent00.obj
 0002:00002c4c       $unwind$?nsk_jni_lverify@@YAHHPEAUJNIEnv_@@HQEBDH1ZZ 0000000180007c4c     libattach009Agent00.obj
 0002:00002c60       $unwind$?nsk_jni_check_exception@@YAHPEAUJNIEnv_@@QEBDH@Z 0000000180007c60     libattach009Agent00.obj
 0002:00002c7c       $unwind$nsk_jvmti_createJVMTIEnv 0000000180007c7c     libattach009Agent00.obj
 0002:00002c90       $unwind$Java_nsk_jvmti_unit_FollowReferences_FollowRefObjects_resetTags 0000000180007c90     libattach009Agent00.obj
 0002:00002c90       $unwind$addRefToVerify     0000000180007c90     libattach009Agent00.obj
 0002:00002c90       $unwind$nsk_aod_internal_error 0000000180007c90     libattach009Agent00.obj
 0002:00002c90       $unwind$nsk_jvmti_resetAgentData 0000000180007c90     libattach009Agent00.obj
 0002:00002c90       $unwind$nsk_jvmti_setFailStatus 0000000180007c90     libattach009Agent00.obj
 0002:00002c90       $unwind$__scrt_initialize_default_local_stdio_options 0000000180007c90     MSVCRT:default_local_stdio_options.obj
 0002:00002c90       $unwind$?dllmain_crt_dispatch@@YAHQEAUHINSTANCE__@@KQEAX@Z 0000000180007c90     MSVCRT:dll_dllmain.obj
 0002:00002c90       $unwind$DllMain            0000000180007c90     MSVCRT:dll_dllmain_stub.obj
 0002:00002c90       $unwind$__GSHandlerCheck   0000000180007c90     MSVCRT:gshandler.obj
 0002:00002c90       $unwind$?__scrt_uninitialize_thread_safe_statics@@YAXXZ 0000000180007c90     MSVCRT:thread_safe_statics.obj
 0002:00002c90       $unwind$__scrt_acquire_startup_lock 0000000180007c90     MSVCRT:utility.obj
 0002:00002c90       $unwind$__scrt_dllmain_after_initialize_c 0000000180007c90     MSVCRT:utility.obj
 0002:00002c90       $unwind$__scrt_dllmain_before_initialize_c 0000000180007c90     MSVCRT:utility.obj
 0002:00002c90       $unwind$__scrt_dllmain_crt_thread_attach 0000000180007c90     MSVCRT:utility.obj
 0002:00002c90       $unwind$__scrt_dllmain_crt_thread_detach 0000000180007c90     MSVCRT:utility.obj
 0002:00002c90       $unwind$__scrt_dllmain_uninitialize_c 0000000180007c90     MSVCRT:utility.obj
 0002:00002c90       $unwind$__scrt_dllmain_uninitialize_critical 0000000180007c90     MSVCRT:utility.obj
 0002:00002c90       $unwind$atexit             0000000180007c90     MSVCRT:utility.obj
 0002:00002c98       $unwind$nsk_jvmti_lverify  0000000180007c98     libattach009Agent00.obj
 0002:00002cac       $unwind$exitOnError        0000000180007cac     libattach009Agent00.obj
 0002:00002cbc       $unwind$Java_nsk_share_jvmti_ArgumentHandler_getAgentOptionsString 0000000180007cbc     libattach009Agent00.obj
 0002:00002cbc       $unwind$nsk_jvmti_aod_deallocate 0000000180007cbc     libattach009Agent00.obj
 0002:00002cd0       $unwind$Java_nsk_jvmti_unit_FollowReferences_FollowRefObjects_getTag 0000000180007cd0     libattach009Agent00.obj
 0002:00002cd0       $unwind$Java_nsk_share_jvmti_DebugeeClass_checkStatus 0000000180007cd0     libattach009Agent00.obj
 0002:00002cd0       $unwind$agentThreadWrapper 0000000180007cd0     libattach009Agent00.obj
 0002:00002ce0       $unwind$nsk_aod_agentLoaded 0000000180007ce0     libattach009Agent00.obj
 0002:00002ce0       $unwind$startAgentThreadWrapper 0000000180007ce0     libattach009Agent00.obj
 0002:00002cfc       $unwind$syncDebuggeeStatus 0000000180007cfc     libattach009Agent00.obj
 0002:00002cfc       $unwind$__scrt_dllmain_exception_filter 0000000180007cfc     MSVCRT:utility.obj
 0002:00002d10       $unwind$Java_nsk_share_jvmti_DebugeeClass_resetAgentData 0000000180007d10     libattach009Agent00.obj
 0002:00002d10       $unwind$nsk_aod_createJNIEnv 0000000180007d10     libattach009Agent00.obj
 0002:00002d18       $unwind$MA_checkStatus     0000000180007d18     libattach009Agent00.obj
 0002:00002d2c       $unwind$Java_nsk_jvmti_unit_FollowReferences_FollowRefObjects_setTag 0000000180007d2c     libattach009Agent00.obj
 0002:00002d44       $unwind$Java_nsk_jvmti_unit_FollowReferences_FollowRefObjects_addRefToVerify 0000000180007d44     libattach009Agent00.obj
 0002:00002d60       $unwind$nsk_aod_createOptions 0000000180007d60     libattach009Agent00.obj
 0002:00002d7c       $unwind$nsk_aod_getOptionValue 0000000180007d7c     libattach009Agent00.obj
 0002:00002d7c       $unwind$nsk_aod_optionSpecified 0000000180007d7c     libattach009Agent00.obj
 0002:00002d90       $unwind$nsk_aod_agentFinished 0000000180007d90     libattach009Agent00.obj
 0002:00002da8       $unwind$nsk_free_options   0000000180007da8     libattach009Agent00.obj
 0002:00002db8       $unwind$nsk_jvmti_aod_disableEventAndFinish 0000000180007db8     libattach009Agent00.obj
 0002:00002dd0       $unwind$nsk_jvmti_aod_getClassName 0000000180007dd0     libattach009Agent00.obj
 0002:00002de4       $unwind$nsk_jvmti_aod_getThreadName 0000000180007de4     libattach009Agent00.obj
 0002:00002dfc       $unwind$classLoadHandler   0000000180007dfc     libattach009Agent00.obj
 0002:00002e1c       $unwind$capture_previous_context 0000000180007e1c     MSVCRT:gs_report.obj
 0002:00002e28       $unwind$__GSHandlerCheckCommon 0000000180007e28     MSVCRT:gshandler.obj
 0002:00002e30       $xdatasym                  0000000180007e30     MSVCRT:amdsecgs.obj
 0002:00002e34       $unwind$?dllmain_crt_process_attach@@YAHQEAUHINSTANCE__@@QEAX@Z 0000000180007e34     MSVCRT:dll_dllmain.obj
 0002:00002e70       $unwind$?fin$0@?0??dllmain_crt_process_attach@@YAHQEAUHINSTANCE__@@QEAX@Z@4HA 0000000180007e70     MSVCRT:dll_dllmain.obj
 0002:00002e70       $unwind$?fin$0@?0??dllmain_crt_process_detach@@YAH_N@Z@4HA 0000000180007e70     MSVCRT:dll_dllmain.obj
 0002:00002e70       $unwind$?fin$1@?0??dllmain_crt_process_detach@@YAH_N@Z@4HA 0000000180007e70     MSVCRT:dll_dllmain.obj
 0002:00002e78       $unwind$?dllmain_crt_process_detach@@YAH_N@Z 0000000180007e78     MSVCRT:dll_dllmain.obj
 0002:00002ecc       $unwind$?dllmain_dispatch@@YAHQEAUHINSTANCE__@@KQEAX@Z 0000000180007ecc     MSVCRT:dll_dllmain.obj
 0002:00002ef4       $unwind$?filt$0@?0??dllmain_dispatch@@YAHQEAUHINSTANCE__@@KQEAX@Z@4HA 0000000180007ef4     MSVCRT:dll_dllmain.obj
 0002:00002efc       $unwind$_DllMainCRTStartup 0000000180007efc     MSVCRT:dll_dllmain.obj
 0002:00002f0c       $unwind$__scrt_is_nonwritable_in_current_image 0000000180007f0c     MSVCRT:utility.obj
 0002:00002f2c       $unwind$__scrt_is_nonwritable_in_current_image$filt$0 0000000180007f2c     MSVCRT:utility.obj
 0002:00002f34       $unwind$__scrt_fastfail    0000000180007f34     MSVCRT:utility_desktop.obj
 0002:00002f44       $unwind$__security_init_cookie 0000000180007f44     MSVCRT:gs_support.obj
 0002:00002f50       $unwind$__isa_available_init 0000000180007f50     MSVCRT:cpu_disp.obj
 0002:00002f60       $xdatasym                  0000000180007f60     MSVCRT:guard_dispatch.obj
 0002:00002f68       $xdatasym                  0000000180007f68     MSVCRT:guard_xfg_dispatch.obj
 0002:00002f70       .edata                     0000000180007f70     attach009Agent00.exp
 0002:00002f98       rgpv                       0000000180007f98     attach009Agent00.exp
 0002:00002fcc       rgszName                   0000000180007fcc     attach009Agent00.exp
 0002:00003000       rgwOrd                     0000000180008000     attach009Agent00.exp
 0002:0000301a       szName                     000000018000801a     attach009Agent00.exp
 0002:0000302f       $N00001                    000000018000802f     attach009Agent00.exp
 0002:0000303e       $N00002                    000000018000803e     attach009Agent00.exp
 0002:00003083       $N00003                    0000000180008083     attach009Agent00.exp
 0002:000030c0       $N00004                    00000001800080c0     attach009Agent00.exp
 0002:00003108       $N00005                    0000000180008108     attach009Agent00.exp
 0002:00003148       $N00006                    0000000180008148     attach009Agent00.exp
 0002:00003185       $N00007                    0000000180008185     attach009Agent00.exp
 0002:000031c0       $N00008                    00000001800081c0     attach009Agent00.exp
 0002:000031ee       $N00009                    00000001800081ee     attach009Agent00.exp
 0002:0000321f       $N00010                    000000018000821f     attach009Agent00.exp
 0002:0000324e       $N00011                    000000018000824e     attach009Agent00.exp
 0002:0000327d       $N00012                    000000018000827d     attach009Agent00.exp
 0002:000032b2       $N00013                    00000001800082b2     attach009Agent00.exp
 0002:000036f2       .idata$6                   00000001800086f2     kernel32:KERNEL32.dll
 0002:00003756       .idata$6                   0000000180008756     vcruntime:VCRUNTIME140.dll
 0002:000038de       .idata$6                   00000001800088de     ucrt:api-ms-win-crt-heap-l1-1-0.dll
 0002:000038fe       .idata$6                   00000001800088fe     ucrt:api-ms-win-crt-runtime-l1-1-0.dll
 0002:00003920       .idata$6                   0000000180008920     ucrt:api-ms-win-crt-stdio-l1-1-0.dll
 0002:00003940       .idata$6                   0000000180008940     ucrt:api-ms-win-crt-string-l1-1-0.dll
 0003:00000000       ?codeAttributeName@@3PEBDEB 0000000180009000     libattach009Agent00.obj
 0003:00000008       ?lineNumberAttributeName@@3PEBDEB 0000000180009008     libattach009Agent00.obj
 0003:00000010       ?localVarAttributeName@@3PEBDEB 0000000180009010     libattach009Agent00.obj
 0003:00000018       ?localVarTypeAttributeName@@3PEBDEB 0000000180009018     libattach009Agent00.obj
 0003:00000020       ?stackMapAttributeName@@3PEBDEB 0000000180009020     libattach009Agent00.obj
 0003:00000028       ?callBytes@@3PAEA          0000000180009028     libattach009Agent00.obj
 0003:0000002c       ?allocBytes@@3PAEA         000000018000902c     libattach009Agent00.obj
 0003:00000030       TARGET_APP_CLASS_NAME      0000000180009030     libattach009Agent00.obj
 0003:00000038       AGENT_LOADED_METHOD_NAME   0000000180009038     libattach009Agent00.obj
 0003:00000040       AGENT_LOADED_METHOD_SIGNATURE 0000000180009040     libattach009Agent00.obj
 0003:00000048       AGENT_FINISHED_METHOD_NAME 0000000180009048     libattach009Agent00.obj
 0003:00000050       AGENT_FINISHED_METHOD_SIGNATURE 0000000180009050     libattach009Agent00.obj
 0003:00000058       success                    0000000180009058     libattach009Agent00.obj
 0003:0001aba0       nsk_context                0000000180023ba0     libattach009Agent00.obj
 0003:0001abac       redefineAttempted          0000000180023bac     libattach009Agent00.obj
 0003:0001abb0       redefineSucceed            0000000180023bb0     libattach009Agent00.obj
 0003:0001abb4       agentFailed                0000000180023bb4     libattach009Agent00.obj
 0003:0001abb8       agentThread                0000000180023bb8     libattach009Agent00.obj
 0003:0001abc0       context                    0000000180023bc0     libattach009Agent00.obj
 0003:0001ac78       agentThreadProc            0000000180023c78     libattach009Agent00.obj
 0003:0001ac80       agentThreadArg             0000000180023c80     libattach009Agent00.obj
 0003:0001ac88       agent_data                 0000000180023c88     libattach009Agent00.obj
 0003:0001ac98       jvmti_env                  0000000180023c98     libattach009Agent00.obj
 0003:0001aca0       jvm                        0000000180023ca0     libattach009Agent00.obj
 0003:0001aca8       jni_env                    0000000180023ca8     libattach009Agent00.obj
 0003:0001acb0       currentAgentStatus         0000000180023cb0     libattach009Agent00.obj
 0003:0001acb4       ?codeAttributeIndex@@3GA   0000000180023cb4     libattach009Agent00.obj
 0003:0001acb8       checkStatus_func           0000000180023cb8     libattach009Agent00.obj
 0003:0001acc0       ?lineNumberAttributeIndex@@3GA 0000000180023cc0     libattach009Agent00.obj
 0003:0001acc4       ?localVarAttributeIndex@@3GA 0000000180023cc4     libattach009Agent00.obj
 0003:0001acc8       ?localVarTypeAttributeIndex@@3GA 0000000180023cc8     libattach009Agent00.obj
 0003:0001accc       ?stackMapAttributeIndex@@3GA 0000000180023ccc     libattach009Agent00.obj
 0003:0001acd0       ?stackFrameOffset@@3GA     0000000180023cd0     libattach009Agent00.obj
 0003:0001acd4       ?mode@@3HA                 0000000180023cd4     libattach009Agent00.obj
 0003:0001acd8       ?orig@@3PEBEEB             0000000180023cd8     libattach009Agent00.obj
 0003:0001ace0       ?gen@@3PEAEEA              0000000180023ce0     libattach009Agent00.obj
 0003:0001ace8       ?inputPos@@3PEAEEA         0000000180023ce8     libattach009Agent00.obj
 0003:0001acf0       ?endPos@@3PEBEEB           0000000180023cf0     libattach009Agent00.obj
 0003:0001acf8       ?genPos@@3PEAEEA           0000000180023cf8     libattach009Agent00.obj
 0003:0001ad00       ?markPos@@3PEAEEA          0000000180023d00     libattach009Agent00.obj
 0003:0001ad08       ?constantPool@@3PEAPEADEA  0000000180023d08     libattach009Agent00.obj
 0003:0001ad10       ?constantPoolSize@@3GA     0000000180023d10     libattach009Agent00.obj
 0003:0001ad14       ?constantPoolCount@@3GA    0000000180023d14     libattach009Agent00.obj
 0003:0001ad18       ?zeroBytes@@3PAEA          0000000180023d18     libattach009Agent00.obj
 0003:0001ad1c       ?codeLength@@3IA           0000000180023d1c     libattach009Agent00.obj
 0003:0001ad20       ?map@@3PEAIEA              0000000180023d20     libattach009Agent00.obj
 0003:0001ad28       ?widening@@3PEACEA         0000000180023d28     libattach009Agent00.obj
 0003:0001ad30       internalError              0000000180023d30     libattach009Agent00.obj
 0003:0001ad34       multiagentsCount           0000000180023d34     libattach009Agent00.obj
 0003:0001ad38       targetAppClass             0000000180023d38     libattach009Agent00.obj
 0003:0001ad40       agentLoadedMethod          0000000180023d40     libattach009Agent00.obj
 0003:0001ad48       agentFinishedMethod        0000000180023d48     libattach009Agent00.obj
 0003:0001ad50       options                    0000000180023d50     libattach009Agent00.obj
 0003:0001ad58       agentName                  0000000180023d58     libattach009Agent00.obj
 0003:0001ad60       disabledForOthers          0000000180023d60     libattach009Agent00.obj
 0003:0001ad70       ?mainThreadName@?1??classLoadHandler@@9@4PADA 0000000180023d70     libattach009Agent00.obj
 0003:0001b170       GS_ExceptionRecord         0000000180024170     MSVCRT:gs_report.obj
 0003:0001b210       GS_ContextRecord           0000000180024210     MSVCRT:gs_report.obj
 0003:0001b6e0       ?g_tss_cv@@3U_RTL_CONDITION_VARIABLE@@A 00000001800246e0     MSVCRT:thread_safe_statics.obj
 0003:0001b6e8       ?g_tss_event@@3PEAXEA      00000001800246e8     MSVCRT:thread_safe_statics.obj
 0003:0001b6f0       ?g_tss_mutex@@3U_RTL_CRITICAL_SECTION@@A 00000001800246f0     MSVCRT:thread_safe_statics.obj
 0003:0001b718       ?g_sleep_condition_variable_cs@@3P6AHPEAU_RTL_CONDITION_VARIABLE@@PEAU_RTL_CRITICAL_SECTION@@K@ZEA 0000000180024718     MSVCRT:thread_safe_statics.obj
 0003:0001b720       ?g_wake_all_condition_variable@@3P6AXPEAU_RTL_CONDITION_VARIABLE@@@ZEA 0000000180024720     MSVCRT:thread_safe_statics.obj
 0003:0001b72c       ?__proc_attached@@3HA      000000018002472c     MSVCRT:dll_dllmain.obj
 0003:0001b740       ?is_initialized_as_dll@@3_NA 0000000180024740     MSVCRT:utility.obj
 0003:0001b741       ?module_local_atexit_table_initialized@@3_NA 0000000180024741     MSVCRT:utility.obj
 0003:0001b748       ?module_local_atexit_table@@3U_onexit_table_t@@A 0000000180024748     MSVCRT:utility.obj
 0003:0001b760       ?module_local_at_quick_exit_table@@3U_onexit_table_t@@A 0000000180024760     MSVCRT:utility.obj
